:100000000C9445010C94BD350C946B0E0C9462015C
:100010000C9462010C9462010C9462010C946201D4
:100020000C9462010C9462010C9462010C94D31044
:100030000C9462010C944C2F0C94862F0C94AF2FCF
:100040000C9462010C9462010C9462010C948A3746
:100050000C94620131313056332E333700000001E9
:100060000000060000FF00000F02000C0014010158
:100070000400001450040100000000000000000013
:1000800000000000010003E8000000000000000381
:10009000E800000000000200FA0600070000FF0070
:1000A0000037060002800000000000002107101049
:1000B0000504030206100D0C0B0A2E1005040302A2
:1000C00006100D0C0B0A2E100504030206100D0C71
:1000D0000B0A2E1111111111111111111111111100
:1000E0001111111111111111111111111111110011
:1000F0000404040808080C0C0C1010101414181830
:10010000181C1C1C20202020242424282828282CCB
:100110002C2C2C30303030343434343438383838B7
:10012000383838383C3C3C3C3C3C3C3C3C3C3C1843
:10013000180B0B0C0C0B0C0B040208040C1803031B
:10014000030801010101010804040101000000008D
:1001500000000C10140808090A0B0C08080C090A06
:100160000B0C0D0E080808090A0A0A0A0A0B0C0CE7
:1001700000010405030647401D1B1C1B14133322FA
:1001800019100C080603016744332219100C0803E8
:10019000524F5200000106524F4C000002064D53D0
:1001A00054000003024D5650000004075341500014
:1001B0000005074741500000060353544150000713
:1001C00003525341500008035347500000090747AA
:1001D000475000000A0353544750000B0352534743
:1001E00050000C0352465300000D0353494F0000CA
:1001F0000E0747494F00000F0353414300001D07FE
:1002000053434F00001E0747434F00001F03434363
:100210004F0000200355463000004007554631008E
:10022000004107554632000042075546330000435F
:10023000075546340000440755463500004507552C
:100240004636000046075546370000470752554ED0
:100250000000810553544F5000800042494E000079
:100260008B0000000000000000535441545553001F
:1002700053544F5000535441525400434F4F524433
:100280000052454C00414253000011241FBECFE5EF
:10029000D8E0DEBFCDBF11E0A0E6B0E0E2E4FBE7CE
:1002A00002C005900D92A431B107D9F717E0A4E17F
:1002B000B1E001C01D92A637B107E1F70E946401C9
:1002C0000C94A03D0C940000EF92FF920F931F93AB
:1002D000CF93DF93CDB7DEB724970FB6F894DEBF88
:1002E0000FBECDBF0E942E0F82E00E94AC100E9474
:1002F000A20F8DB18F738DB981E887BB30E020E00C
:1003000018BA00000000000096B380E888BB000027
:1003100000000000B69B02C096FF2F5F3F5F3A309F
:1003200079F72A3039F560E089E090E00E941910F1
:1003300060E080E090E00E9419101A82198205C0E6
:1003400089819A8101969A83898389819A818F5FB5
:100350009F4FB1F7C0981A82198205C089819A818E
:1003600001969A83898389819A818F5F9F4FB1F724
:10037000C09AE3CF0E942E0F82E00E94AC100E9430
:100380007D0E0E942E110E94A20FAB980E946F0F4B
:100390000E94850F80E090E00E941110843E09F4D5
:1003A000DBC0C0980E946B3060E089E090E00E9462
:1003B000191040E16DE570E080E090E00E945E1071
:1003C00061E08AE491E00E94191060E08BE491E022
:1003D0000E94191060E08CE491E00E94191060E026
:1003E0008DE491E00E94191062E08EE491E00E9499
:1003F000191060E08FE491E00E94191060E080E540
:1004000091E00E94191060E081E591E00E941910CE
:100410000E9436104DE26CE770E08DE390E00E94A0
:100420005E104DE26CE770E08AE690E00E945E109C
:100430004DE26CE770E087E990E00E945E1043E0D7
:1004400069EA70E084EC90E00E945E1043E06CEAA0
:1004500070E087EC90E00E945E1040E86FEA70E088
:100460008AEC90E00E945E1064E68AE591E00E94CA
:10047000191060E08BE591E00E94191064E68CE5AC
:1004800091E00E94191060E08DE591E00E94191042
:1004900064E68EE591E00E94191060E08FE591E03E
:1004A0000E94191060E080E691E00E94191060E05F
:1004B00081E691E00E94191060E082E691E00E94DE
:1004C000191060E083E691E00E94191060E084E674
:1004D00091E00E94191060E085E691E00E941910F9
:1004E00060E08DEF93E00E94191060E08EEF93E0E2
:1004F0000E94191060E08FEF93E00E94191060E0F5
:1005000086E691E00E94191068E087E691E00E947B
:10051000191060E088E691E00E94191068E089E611
:1005200091E00E94191060E08AE691E00E941910A3
:1005300068E08BE691E00E94191081E090E00E9453
:100540001110EEE5F0E0E4918E1729F464EE80E0FE
:1005500090E00E941910C09A81E090E00E94111072
:100560000E94C42F8AE090E00E9411108093C10481
:10057000882311F00E948E388EE70E944E0B00E017
:10058000802F80610E944E0B802F88610E944E0B4D
:10059000802F84600E944E0B802F86600E944E0B3D
:1005A000802F84610E944E0B005E003649F70E9446
:1005B000CD090E948610EE24FF24C70125E0880F94
:1005C000991F2A95E1F78D600E94E30F082F10E034
:1005D000C80101960E9411108C83C80102960E94E6
:1005E00011108B836B817C818E2D0E948908C7013D
:1005F00085960E941110682F8E2D0E94E00F08949E
:10060000E11CF11C83E0E816F104B9F62FEF4FEF7F
:1006100060E086E10E94E9052FEF4FEF60E086E39E
:100620000E94E9052FEF4FEF60E086E50E94E905A3
:100630008AE491E00E941110809335078BE491E0E9
:100640000E941110809336078CE491E00E941110F3
:10065000809337078DE491E00E9411108093380752
:100660008EE491E00E9411108093ED068FE491E0FA
:100670000E9411108093EE0680E591E00E94111017
:100680008093EF0681E591E00E9411108093F006BF
:10069000E0903507F0903607009137071091380742
:1006A00085E090E00E941110B801A70190E00E943F
:1006B000B6348AE591E00E941110809316078BE50D
:1006C00091E00E941110809317078CE591E00E9441
:1006D0001110809318078DE591E00E94111080930E
:1006E00019078EE591E00E94111080931A078FE59B
:1006F00091E00E94111080931B0780E691E00E9418
:1007000011108093F80681E691E00E941110809309
:10071000F90682E691E00E9411108093FA0683E6C2
:1007200091E00E9411108093FB0684E691E00E9404
:1007300011108093FC0685E691E00E9411108093D1
:10074000FD068DEF93E00E94111080931D078EEF40
:1007500093E00E94111080931E078FEF93E00E9498
:10076000111080931F0786E691E00E94111080937C
:100770005B0187E691E00E94111080935C0188E69E
:1007800091E00E94111080935D0189E691E00E9442
:10079000111080935E018AE691E00E94111080930F
:1007A0005F018BE691E00E9411108093600182E06E
:1007B00090E00E9411100E944B3783E090E00E946D
:1007C000111080FF03C082E08093620183E090E01B
:1007D0000E94111082958F70809363010E94CB2E2E
:1007E0000E94FE0378940E94A7060E9434110E9482
:1007F000840B0E9462290E940404F5CF81E080935B
:10080000D5051092B60608958091390781FF07C07B
:100810008091B6068F3F19F08F5F8093B606809166
:10082000D505813051F48091B6068F3030F0C098F4
:100830001092B60682E08093D5058091D50582306E
:1008400051F48091B606853030F0C09A1092B60609
:1008500081E08093D5050895089508950895089539
:10086000089508950895CF92DF92EF92FF920F932B
:100870001F93CF93DF93CDB7DEB729970FB6F894C8
:10088000DEBF0FBECDBF82E00E945B118CE090E026
:100890000E941110898382E090E00E9411108A83E7
:1008A00081E88B8381E48C838091D2068D83809153
:1008B000D1068E838091D3068F838091D506888759
:1008C00019868E010F5F1F4F680189E0E82EF12C19
:1008D000EC0EFD1E8985F8019081890F8987809132
:1008E0006201882319F480810E9410300F5F1F4F2E
:1008F0000E151F0579F780916201882319F4898507
:100900000E94103080916201882319F0C6010E9474
:10091000813929960FB6F894DEBF0FBECDBFDF91A7
:10092000CF911F910F91FF90EF90DF90CF9008959E
:10093000682F70E080FD2FC0CB018076907035E08D
:10094000959587953A95E1F7E82FCB018F799070CF
:100950008431910529F4F0E0EE5CF84F208308958E
:100960008630910541F4F0E0EE0FFF1FE552F94F9C
:10097000208341830895089771F4F0E0EE0FFF1F84
:10098000E45DF84F2083418343FF05C0808191815E
:10099000906F918380830895EF92FF920F931F933E
:1009A000182F062FF42EE22E0E9498048BB78F7B0F
:1009B0008BBFC398812F0E94BB10802F0E94BB1059
:1009C0008F2D0E94BB108E2D0E94BB10C39A8BB737
:1009D00080648BBF1F910F91FF90EF900895CF928D
:1009E000DF92EF92FF920F931F93CF93DF937C01DF
:1009F0006B01DC018C9190E09C012F793070211506
:100A0000310519F02830310501F5EC01C076D070C0
:100A100045E0D595C7954A95E1F7C330B0F48C2FE2
:100A20008B5E0E949810682F8C2F0E94E00FEC2F95
:100A3000F0E09F012353394FDF01A05ABF4F8C9143
:100A4000D9018C93E050F94F1082F7012381428144
:100A5000618180810E9498048BB78F7B8BBFC39884
:100A6000C0E0D0E086010C0F1D1FF701EC0FFD1F49
:100A700080810E94BB10D8018C932196C430D1058F
:100A800089F7C39A8BB780648BBF80E090E0DF91D9
:100A9000CF911F910F91FF90EF90DF90CF9008952D
:100AA0005F926F927F928F929F92AF92BF92CF92FE
:100AB000DF92EF92FF920F931F93CF93DF93CDB707
:100AC000DEB728970FB6F894DEBF0FBECDBF282F34
:100AD00030E0F901E653F94F8081882319F4662349
:100AE00009F461C060831A82C901880F991F820FBF
:100AF000931F880F991F880F991FF0E85F2E580EDB
:100B000000E010E0862F90E0E4E0AE2EB12CA822A9
:100B1000B92272E0C72ED12CC822D92261E0E62E7C
:100B2000F12CE822F92255E0652E712C6C0E7D1E09
:100B30004E010894811C911CA114B10489F0063067
:100B400020F4E114F10421F006C0C114D10419F419
:100B500090E180E102C091E181E18B839C830CC034
:100B6000C80185539F4F0E9411108B83C801865383
:100B70009F4F0E9411108C83902F002311F006309C
:100B800011F480E18C839A3019F48B8180628B831D
:100B9000950D9983B301C4010E94EF040E5F1F4FAE
:100BA0000C30110549F628960FB6F894DEBF0FBE3B
:100BB000CDBFDF91CF911F910F91FF90EF90DF900C
:100BC000CF90BF90AF909F908F907F906F905F90ED
:100BD00008953F924F925F926F927F928F929F9271
:100BE000AF92BF92CF92DF92EF92FF920F931F933B
:100BF000CF93DF93CDB7DEB728970FB6F894DEBF5B
:100C00000FBECDBFC82E562E442E322E90E09C0132
:100C10002F7930702115310521F02830310509F088
:100C200064C08076907045E0959587954A95E1F788
:100C3000D82E82E08D1508F458C0ED2CFF24F70162
:100C4000EE0FFF1FDF01A850B94F8D919C91EE5A16
:100C5000FE4F91838083F701E85AFE4F80818823FD
:100C600071F110821A828CE0D89EC00111248C018F
:100C700000581F4F2CE8A22EB12CA80EB91E85E0FB
:100C8000682E712C6C0E7D1E4E010894811C911CE7
:100C900013C00983C801855B9F4F0E9411108B838D
:100CA000C801865B9F4F0E9411108C83B301C40161
:100CB0000E94EF040E5F1F4F0A151B0550F38D2D88
:100CC0008B5E0E949810682F8D2D0E94E00FD70137
:100CD000A353B94FF701E05AFF4F80818C93E0E0B6
:100CE000F7E0EE0EFF1EF7011082232D442D652D37
:100CF0008C2D0E9498048BB78F7B8BBFC3988C2D53
:100D00000E94BB10852D0E94BB10842D0E94BB1039
:100D1000832D0E94BB10C39A8BB780648BBF28962B
:100D20000FB6F894DEBF0FBECDBFDF91CF911F91FC
:100D30000F91FF90EF90DF90CF90BF90AF909F907A
:100D40008F907F906F905F904F903F900895AF92FB
:100D5000BF92CF92DF92EF92FF920F931F93CF93A8
:100D6000DF93CDB7DEB72A970FB6F894DEBF0FBE7C
:100D7000CDBF1092BF061092C0061092C10680919E
:100D8000C806882311F083995FC0809114018F5F9A
:100D900080931401833010F0109214018EE090E0E3
:100DA0000E9411108F5F8093C80680911401829574
:100DB000880F807E8B608F838E010D5F1F4F67E0F1
:100DC000C62ED12CCC0EDD1EB801C6010E94EF0448
:100DD0008B818093C9068D8183FF02C0806F8D83D4
:100DE0008D818A838E818983E0911401F0E0EE0F7A
:100DF000FF1FEE53F94F89819A81918380838399F4
:100E000023C0EE24FF2458011E2D1295110F107ED1
:100E1000812F87618F83B501C6010E94EF04F7011E
:100E2000E154F94F8E81808316611F838FEF89878C
:100E30008A87B501C6010E94EF040894E11CF11CE9
:100E400083E0E816F10401F72A960FB6F894DEBFA6
:100E50000FBECDBFDF91CF911F910F91FF90EF900B
:100E6000DF90CF90BF90AF900895CF93DF93EC01C8
:100E700082E090E00E94111080932801909125015A
:100E8000992359F08091390780FF03C091509093C6
:100E900025018091240181600EC080912701882363
:100EA00039F0809124018061809324011092270100
:100EB000809124018E7F80932401809127018823D3
:100EC000F1F585E191E00E94E5338823C1F120919D
:100ED00018013091190140911A0150911B01809124
:100EE000350790913607A0913707B091380728173A
:100EF00039074A075B0719F580911501873008F417
:100F000080C09E01295F3F4F809128018F83ECE1D3
:100F1000F1E0DE0180818D93E90188819191890F53
:100F2000888381E0E332F807A9F7809115018730C3
:100F300011F481E001C082E08093E5066DC08091EC
:100F40002701882379F468E0CE010E94573788236F
:100F500049F08F8190912801890F8F8381E08093E0
:100F60001C075AC00E94EC2F8F3F31F4809124015E
:100F70008061809324013AC089E291E00E942C3084
:100F80008130A1F584E1809325012091270122235E
:100F900029F4809129018093260125C09091260192
:100FA000809128019817D1F430912401932F9460F7
:100FB0009093240191FD12C0C20FD11D2197809101
:100FC00029018883283051F494FF04C09F7E9093B8
:100FD000240106C036603093240102C0283018F086
:100FE0001092270103C02F5F209327011092E5067E
:100FF00010921C078091240184FF06C08F7E80938D
:1010000024018FEF9FEF0AC081FD03C080E090E0D4
:1010100005C08D7F8093240181E090E0DF91CF9126
:101020000895FB0120813181280F391F35952795BF
:1010300031832083C9010895FF920F931F93F62EE9
:1010400081608093E10606EE16E0B80181EE96E03D
:101050000E94EF040F0D111DF801808190E01F9197
:101060000F91FF90089581608093E10666EE76E02F
:1010700081EE96E00E94EF048091E90690E00895E9
:1010800081608093E10666EE76E081EE96E00E9454
:10109000EF042091E80630E0522F44278091E906C2
:1010A00090E0482B592B23FD02C0CA010895CA01C4
:1010B000906F0895CF93DF93CDB7DEB724970FB627
:1010C000F894DEBF0FBECDBF81608093E10666EE6F
:1010D00076E081EE96E00E94EF049091E70697FF9C
:1010E00003C08FEF8C8301C01C829B838091E80634
:1010F0008A838091E906898369817A818B819C81C9
:1011000024960FB6F894DEBF0FBECDBFDF91CF910E
:101110000895CF92DF92FF920F931F93CF93DF93A7
:10112000CDB7DEB721970FB6F894DEBF0FBECDBFA7
:101130008B01F82EF294FF0C70EEF7228F2D89614F
:101140008093E10666EE76E081EE96E00E94EF0481
:10115000C8018070987F892B19F08FEF9FEF57C0DF
:101160008091E806982F9F709C5F82958F70981BE6
:101170000F3F1105F9F0F4F06801191694F0412FB2
:101180005527202F60E08F2D8C600E94E90520E01C
:101190004FE760E08F2D82610E94E90581E090E0D9
:1011A00036C0D594C79491508FEFC816D104E1F0A2
:1011B000DCF0E3CF68019D3094F0412F5527202FBC
:1011C00060E08F2D8C600E94E9052DE040E060E03A
:1011D0008F2D82610E94E90582E090E018C0CC0C5E
:1011E000DD1C9F5FC7FEE7CF412F5527202F60E012
:1011F0008F2D8C6099830E94E9059981292F4C2DB0
:1012000060E08F2D82610E94E90580E090E02196E8
:101210000FB6F894DEBF0FBECDBFDF91CF911F9107
:101220000F91FF90DF90CF9008950F931F93062F9B
:10123000182F1295110F107E812F85618093E10682
:1012400066EE76E081EE96E00E94EF04202F40915A
:10125000E80660E0812F84610E94E9051F910F91EB
:101260000895CF93DF93CDB7DEB724970FB6F894E8
:10127000DEBF0FBECDBF49835A836B837C83298138
:101280004A816B810E94E90524960FB6F894DEBF6F
:101290000FBECDBFDF91CF9108951F93182F62E04D
:1012A0000E9415091295110F107E40E050E060E099
:1012B00070E0812F88600E94310940E050E060E0DA
:1012C00070E0812F8A600E9431091F9108958295F4
:1012D000880F807E40E050E060E070E088600E940F
:1012E00031090895E82FF0E0EE0FFF1FED59F84F98
:1012F00040815181662329F002C0559547956A9532
:10130000E2F7509541955F4F662757FD6095762F20
:101310008295880F807E88600E9431090895E82FA9
:10132000F0E0EE0FFF1FED59F84F40815181662329
:1013300029F002C0559547956A95E2F7662757FD53
:101340006095762F8295880F807E88600E94310993
:1013500008950F931F93CF93DF93CDB7DEB72297F6
:101360000FB6F894DEBF0FBECDBF8C0101970E946F
:101370001110FE0131968183C8010E9411108983EA
:1013800089819A8122960FB6F894DEBF0FBECDBF39
:10139000DF91CF911F910F910895CF92DF92EF923D
:1013A000FF920F931F93CF93DF93CDB7DEB72897AC
:1013B0000FB6F894DEBF0FBECDBF1A820BEC10E063
:1013C00085E0C82ED12CCC0EDD1E7E010894E11CD8
:1013D000F11C802F8B548983C8010E9411108B83CC
:1013E000C80101970E9411108C83B601C7010E94A9
:1013F000EF040E5F1F4F81E00B34180751F728965A
:101400000FB6F894DEBF0FBECDBFDF91CF911F9115
:101410000F91FF90EF90DF90CF9008951F939091E0
:10142000300180912F01981719F480E090E040C0BE
:10143000E92FF0E0EB5BFE4F1081892F8F5F8093E7
:1014400030018A3011F410923001E3E2F7E011929A
:1014500087E0EC32F807D9F78CE090E00E94111099
:101460008093230782E090E00E941110809324076C
:1014700080E8809325078AE88093260710932A073F
:1014800020912107233019F4E4E2F7E005C08091B0
:10149000230780932B07F8CF819190912B07890F19
:1014A00080932B0787E0EB32F807B1F7822F90E0AB
:1014B0001F910895EF92FF920F931F938B01E82ED7
:1014C000FF24C70125E0880F991F2A95E1F788615D
:1014D0000E943308877002C0000F111F8A95E2F73F
:1014E000612F772767FD7A95C7014C960E941910E6
:1014F000602FC7014F960E9419101F910F91FF9006
:10150000EF900895CF92DF92EF92FF920F931F9387
:10151000CF93DF93CDB7DEB728970FB6F894DEBF31
:101520000FBECDBF1A820BE011E035E0C32ED12CE7
:10153000CC0EDD1E7E010894E11CF11C802F8A5424
:101540008983B601C7010E94EF046F81C8010E9420
:1015500019106885C80101970E9419100E5F1F4F6E
:1015600081E00B34180751F728960FB6F894DEBFC8
:101570000FBECDBFDF91CF911F910F91FF90EF90E4
:10158000DF90CF900895CF92DF92EF92FF920F936A
:101590001F93CF93DF93CDB7DEB728970FB6F8949C
:1015A000DEBF0FBECDBF1A820BEC10E045E0C42EAB
:1015B000D12CCC0EDD1E7E010894E11CF11C802F85
:1015C0008A548983B601C7010E94EF046F81C80164
:1015D0000E9419106885C80101970E9419100E5FBA
:1015E0001F4F81E00B34180751F728960FB6F89477
:1015F000DEBF0FBECDBFDF91CF911F910F91FF9046
:10160000EF90DF90CF9008950F931F93CF93DF93C8
:10161000082F816007FD24C08093E10666EE76E026
:1016200081EE96E00E94EF04802F0E94E30FC6EE49
:10163000D6E0002711270C1B1D0B080F111D698117
:10164000C8018C0F9D1F0E941910823019F482E08E
:1016500090E01FC0219686E0C93ED80781F717C0E9
:101660008093E10666EE76E081EE96E00E94EF045C
:1016700010E06091E806C801855B9F4F0E94191039
:101680006091E906C801865B9F4F0E94191080E0B7
:1016900090E0DF91CF911F910F910895FF920F93EA
:1016A0001F93CF93DF93CDB7DEB728970FB6F8948B
:1016B000DEBF0FBECDBFF82E0E94E30F082F10E053
:1016C000F982C8010E9411108A83C80101960E9404
:1016D00011108B83C80102960E9411108C83BE01E9
:1016E0006B5F7F4FCE0101960E94EF0480E090E097
:1016F00028960FB6F894DEBF0FBECDBFDF91CF9115
:101700001F910F91FF9008952F923F924F925F92F9
:101710006F927F928F929F92AF92BF92CF92DF9201
:10172000EF92FF920F931F93CF93DF93CDB7DEB766
:1017300024970FB6F894DEBF0FBECDBF86E090E0D1
:101740000E9411108A83809141018F5F8093410133
:101750008150823010F01092410180912A0188233B
:1017600069F480E68093E10666EE76E081EE96E02D
:101770000E94EF0410922B0181E01BC08130E1F444
:1017800081E68093E10666EE76E081EE96E00E94C7
:10179000EF048091E60686FD72C08091E80686958A
:1017A000809587708093EA068091E906809303070D
:1017B00082E080932A0163C0823009F060C080918A
:1017C0002B01A82FB0E0FD01E35EF84F9081992333
:1017D00009F450C0FD01E651F94F8081891708F4E2
:1017E00049C015E0AA0FBB1F1A95E1F78A2F8A603E
:1017F0000E944008BC01892B09F43FC0A0912B0135
:101800004A2F50E0FA01EE5CF84F8081FA01EE0FAA
:10181000FF1F882319F0E45DF84F02C0E552F94F2D
:1018200020813181CB0177FF03C0909581959F4F37
:1018300037FF03C0309521953F4F82179307E9F496
:10184000FA01EE5BFE4F8081823078F08A2F0E9491
:101850004D09E0912B01F0E0DF01A050B94F81E08C
:101860008C93EE5BFE4F108208C08F5F80831092D6
:101870002A0103C0AE5BBE4F1C9210922A018091D8
:10188000390780FFAFC180E00E94A03181E00E9453
:10189000A03182E00E94A0318DE78093E10666EEE0
:1018A00076E081EE96E00E94EF0410913001E09125
:1018B0002F0170916101A0E0B0E041E050E00A2EFC
:1018C00002C0440F551F0A94E2F7642F842F872328
:1018D000D9F08091E60690E09D01220F331F02C0EF
:1018E000959587952A95E2F780FF0EC08E2F8F5F22
:1018F0008A3009F480E0811729F0F0E0EB5BFE4FBD
:101900004083E82F609576231196A330B105A9F6A0
:10191000E0932F01709361018091390781FFAEC080
:101920000FE411E0E8E56E2EE1E07E2E7CE2872EEA
:1019300071E0972E66E1462E67E0562E5DECA52EEF
:1019400056E0B52E1C821B8240E8C42E36E8332EAA
:10195000DB808B819C8125E0880F991F2A95E1F718
:101960008A600E9440087C01F5018081E114F10445
:1019700081F0882341F48D2D8B5E0E949810682F92
:101980008B810E94E00FEB81FC81E05AFF4F808148
:101990000BC0882341F48B810E949810682F8B81A3
:1019A0000E94E00F03C08150F5018083F201208185
:1019B0003181FFEF2F3F3F07A9F4F801808182308A
:1019C00009F441C021E145E060E08C2D0E94CC0487
:1019D00021E14DE060E0832D0E94CC0482E0F8011B
:1019E000808331C0C701F7FE03C0909581959F4F5A
:1019F000F80140818217930794F0413021F127E0EC
:101A000045E060E08C2D0E94CC042FE04DE060E0CA
:101A1000832D0E94CC0481E0F801808310C0442310
:101A200091F020E145E060E08C2D0E94CC0420E1A3
:101A30004DE060E0832D0E94CC04F8011082F30198
:101A40001082F40110828B819C8101969C838B8390
:101A50009CE0C90E390E0F5F1F4F0894611C711C6A
:101A60000894811C911CE2E0F0E04E0E5F1E089489
:101A7000A11CB11CF4EACF1609F06ACF88EF282E1A
:101A800086E0382E0CE2C02E01E0D02E1BE5412E60
:101A900011E0512EB8E56B2EB1E07B2EA2E58A2E27
:101AA000A1E09A2EAA24BB248AE88983C501F5E027
:101AB000880F991FFA95E1F78A600E9440087C011F
:101AC00097FF04C0F094E194F108F394F101808150
:101AD0009181892B39F1E114F10421F5F401808120
:101AE00091810097D9F4F30180818823D9F4198179
:101AF0001A5000E020E140E160E0812F0E94CC0418
:101B00000E5F1E5F0C30B1F720E140E360E0898199
:101B10000E94CC0481E0F301808304C00197F401AA
:101B200091838083AA2009F044C0F20180819181D1
:101B3000009709F4AFC0E816F90608F4ABC0F60147
:101B40008081882309F0A6C081E0808300EC10E04A
:101B50002CE24CE260E0802F0E94CC040E5F1F4F0D
:101B6000F1E000301F0709F495C0F2CF892B09F589
:101B7000F60180818823E9F01082EAE0EE2EE1E0B0
:101B8000FE2EC7010E941110182FC70101960E9456
:101B90001110212F482F60E08E2D8A540E94CC0412
:101BA00082E090E0E80EF91E9AE4E91691E0F90669
:101BB00041F70894A11CB11CE2E0F0E02E0E3F1E9C
:101BC0000894C11CD11C4E0E5F1EF981F45FF9838D
:101BD0000894611C711C82E090E0880E991EFE3A08
:101BE00009F064CF8091D0068823F9F484E08093D3
:101BF000D00668E086E097E00E94890FA7B1B0E0C8
:101C0000AA0FBB1FAF5CBE4FE7B1F0E0EE0FFF1FA6
:101C1000EA5FF84F8D919C91119720813181820F5D
:101C2000931F959587958D939C9390914101E92FF2
:101C3000F0E0EB50F94F8081882319F0892F0E9442
:101C4000AE319A81992311F1EA81E13019F49A9920
:101C500006C01CC0FA81F230C9F49A9917C0AB9A39
:101C600081E08093200700E010E062E0802F0E9476
:101C70001509802F0E946709F801EB50F94F108277
:101C80000F5F1F4F0330110569F0EFCFAB98109233
:101C9000200708C0F20180819181E816F90608F456
:101CA00067CF64CF24960FB6F894DEBF0FBECDBFCA
:101CB000DF91CF911F910F91FF90EF90DF90CF9028
:101CC000BF90AF909F908F907F906F905F904F905C
:101CD0003F902F9008951F920F920FB60F921124EC
:101CE0008F9381E08093D4068F910F900FBE0F9059
:101CF0001F9018951092D40608951F93CF93DF93E9
:101D0000CDB7DEB722970FB6F894DEBF0FBECDBFBA
:101D100023E040E060E084E10E94CC0423E040E066
:101D200060E084E30E94CC0423E040E060E084E5CE
:101D30000E94CC0420E040E060E08AE00E94CC04F5
:101D400020E040E060E08AE20E94CC0420E040E035
:101D500060E08AE40E94CC0410E002C01431A1F0DB
:101D600020E040E060E0812F0E94CC0420E040E0D1
:101D700060E0812F80620E94CC0420E040E060E0BF
:101D8000812F80640E94CC041E5F1C3138F320E058
:101D900040E060E08EE70E94CC0410E020E040E0EC
:101DA00060E0812F80680E94CC041E5F1038B1F77C
:101DB0002FEF47E060E08AE00E94CC041A8219828B
:101DC00006C0000089819A8101969A83898389815E
:101DD0009A81885B9B40ACF320E040E060E08AE0C1
:101DE0000E94CC048BB78F7B8BBFC39883E00E948B
:101DF000BB1080E00E94BB108093D80680E00E9458
:101E0000BB108093D70680E00E94BB108093D6065B
:101E1000C39A8BB780648BBF20E040E060E082E033
:101E20000E94CC048091D6069091D706A091D80646
:101E3000B091D906805D9740A040B04010F480E199
:101E400001C088E08093DA0622960FB6F894DEBFD0
:101E50000FBECDBFDF91CF911F910895CF93DF9338
:101E6000CDB7DEB722970FB6F894DEBF0FBECDBF59
:101E70008EEF8ABB8CE08BBB8DEB87BB8FE188BB81
:101E80008CEF84BB83EF85BB82EF81BB85E082BB97
:101E9000DB981A82198206C0000089819A81019616
:101EA0009A83898389819A8184369105ACF3DB9A80
:101EB0001A82198206C0000089819A8101969A834C
:101EC000898389819A8184369105ACF322960FB675
:101ED000F894DEBF0FBECDBFDF91CF91089581B3DF
:101EE000806B81BB81EF8FBD81E08EBD81E785BDB9
:101EF0000895882319F41BBC6ABD0895813019F434
:101F000019BC68BD089563BD089517B886EC86B9FD
:101F10000895E7B1F0E0EE0FFF1FE80FF91F84B15D
:101F200095B19183808387B190E070E061507040FB
:101F30008617970724F487B18F5F87B901C017B858
:101F4000369A08950895882309F4D99A0895882324
:101F500009F4D9980895882319F080E090E0089555
:101F600089B390E0817090700895482F662359F0EE
:101F70002BB381E090E002C0880F991F4A95E2F7E9
:101F8000282B2BBB08952BB381E090E002C0880F73
:101F9000991F4A95E2F7809582238BBB0895882389
:101FA00019F080E090E008958BB390E096958795C6
:101FB0008170907008958BBB089580E090E0089543
:101FC0000E94790F0895282F87FD23C0482F46953A
:101FD0004F7083E0489FC001112430E020763070BC
:101FE0002115310511F4CD961AC02032310519F4AE
:101FF00086599F4F14C02034310519F489569F4FDC
:102000000EC04F3019F487EC90E009C04E3039F41F
:1020100004C0265B822F90E0089583E090E090E07A
:102020000895DC01E199FECF0E94523D802D90E0A1
:1020300008951F93CF93DF93EC01162F89E090E072
:102040000E941110882331F0C930D10519F082E0C7
:1020500090E008C0E199FECFDE01012E0E945A3DBA
:1020600080E090E0DF91CF911F910895EF92FF9271
:102070001F93CF93DF938DE6E82E80E0F82EC0E12A
:10208000D0E0F7011491612FCE010E941910612F49
:10209000CE0101960E941910612FCE0102960E9476
:1020A00019100894E11CF11C2396CD33D10549F792
:1020B000DF91CF911F91FF90EF900895CF92DF9223
:1020C000EF92FF920F931F93CF93DF936C017B01ED
:1020D000042F10E0C0E0D0E00CC0FE01EE0DFF1DAB
:1020E000E4916E2FCE018C0D9D1D0E9419101F5F73
:1020F0002196101791F780E090E0DF91CF911F912A
:102100000F91FF90EF90DF90CF900895CF93DF93E2
:10211000C0E1D0E0CE010E941110FE01EC5AFE4F4A
:1021200080832196CD33D105A9F7DF91CF91089512
:10213000E4E6F1E0E80FF11D808190E008958D3232
:1021400018F081E090E00895E82FF0E0EC59FE4FA0
:10215000608380E090E0089583708DB98DB18C65C7
:102160008DB9709A10929101089580919101109209
:10217000910190E008958FB980E009C0893C31F465
:102180008091910181608093910103C08F5F779B63
:10219000F5CF769B05C0809191018260809391017B
:1021A0008FB190E008951F920F920FB60F921124F5
:1021B0008F939F93AF93BF938091DA06883011F489
:1021C00082E701C083E282BF80913A07882319F039
:1021D000815080933A078091C806882319F0815076
:1021E0008093C80680919501882321F081508093C7
:1021F00095012BC088E080939501809192018823FE
:1022000019F08150809392018091D006882319F0B3
:1022100081508093D0068091F1069091F206A091B2
:10222000F306B091F4060196A11DB11D8093F1064D
:102230009093F206A093F306B093F4068091FE0605
:10224000882319F081508093FE06BF91AF919F9132
:102250008F910F900FBE0F901F90189582E083BF53
:1022600081E089BF88BF089510923907809192015B
:10227000882301F59AE09093920181E080933907D9
:1022800080919301882321F08150809393010895D8
:102290009093930183E08093390780919401882380
:1022A00021F081508093940108959093940187E0E8
:1022B0008093390708958093C401089599E0699F38
:1022C000A001112490E0837090709C01220F331FB5
:1022D000280F391F420F531F455E5D4F82E0403D7E
:1022E000580714F04BE152E0CA0108950F931F9371
:1022F000CF93DF93CDB7DEB728970FB6F894DEBF44
:102300000FBECDBFE82F0D831E832F8338878093A8
:10231000750760933F074093400781E08093610712
:1023200038853093D2062F812093D1069E819093D9
:10233000D3068D818093D5069093BC018093BB0119
:102340003093C0012093BF019093BE018093BD01E3
:10235000F0E0EE0FFF1FED59FF4F0190F081E02DEF
:102360008091F001811109958091D20687FF03C009
:102370008FEF8C8301C01C828091D1068B8380916A
:10238000D3068A838091D506898369817A818B817E
:102390009C8128960FB6F894DEBF0FBECDBFDF91AB
:1023A000CF911F910F9108950000089500000895A6
:1023B000000008950000089580913F078823A9F444
:1023C0008091480790914907A0914A07B0914B0727
:1023D0002091BD013091BE014091BF015091C001DB
:1023E000820F931FA41FB51FC4C08130A9F4809130
:1023F000480790914907A0914A07B0914B07209157
:10240000BD013091BE014091BF015091C001821BBE
:10241000930BA40BB50BADC0823099F460914807C3
:102420007091490780914A0790914B072091BD0117
:102430003091BE014091BF015091C0010E94C73C44
:1024400031C08330D9F46091480770914907809179
:102450004A0790914B072091BD013091BE014091F8
:10246000BF015091C0010E940D3D20934807309359
:10247000490740934A0750934B0783C08430D9F4EF
:10248000609148077091490780914A0790914B07E6
:102490002091BD013091BE014091BF015091C0011A
:1024A0000E940D3D609348077093490780934A0747
:1024B00090934B0766C08530A9F4809148079091AE
:1024C0004907A0914A07B0914B072091BD01309177
:1024D000BE014091BF015091C00182239323A423E8
:1024E000B52347C08630A9F48091480790914907E9
:1024F000A0914A07B0914B072091BD013091BE01D8
:102500004091BF015091C001822B932BA42BB52B7E
:1025100030C08730A9F48091480790914907A09175
:102520004A07B0914B072091BD013091BE01409107
:10253000BF015091C00182279327A427B52719C056
:10254000883069F48091480790914907A0914A0723
:10255000B0914B0780959095A095B0950AC08930B1
:1025600081F48091BD019091BE01A091BF01B09115
:10257000C0018093480790934907A0934A07B093FE
:102580004B078091480790914907A0914A07B09165
:102590004B072091C6013091C7010097A105B105F5
:1025A00011F4286001C0277F3093C7012093C60132
:1025B000089580913F078823A9F48091480790915E
:1025C0004907A0914A07B0914B07209171073091BC
:1025D00072074091730750917407820F931FA41FD5
:1025E000B51F16C08130E9F48091480790914907E2
:1025F000A0914A07B0914B07209171073091720763
:102600004091730750917407821B930BA40BB50B79
:102610008093480790934907A0934A07B0934B07CC
:10262000D8C0823099F46091480770914907809131
:102630004A0790914B0720917107309172074091A2
:102640007307509174070E94C73C31C08330D9F49E
:10265000609148077091490780914A0790914B0714
:102660002091710730917207409173075091740760
:102670000E940D3D209348073093490740934A0735
:1026800050934B07A6C08430D9F4609148077091ED
:10269000490780914A0790914B072091710730912B
:1026A000720740917307509174070E940D3D60932B
:1026B00048077093490780934A0790934B0789C056
:1026C0008530A9F48091480790914907A0914A0765
:1026D000B0914B07209171073091720740917307B9
:1026E0005091740782239323A423B52391CF86307E
:1026F000A9F48091480790914907A0914A07B091A9
:102700004B072091710730917207409173075091E8
:102710007407822B932BA42BB52B7ACF8730A9F487
:102720008091480790914907A0914A07B0914B07C3
:10273000209171073091720740917307509174078F
:1027400082279327A427B52763CF883069F4809127
:10275000710790917207A0917307B09174078095EB
:102760009095A095B0950AC0893089F4809148076A
:1027700090914907A0914A07B0914B078093710748
:1027800090937207A0937307B093740722C08A30A6
:1027900001F5209148073091490740914A0750912F
:1027A0004B078091710790917207A0917307B091C8
:1027B00074078093480790934907A0934A07B09302
:1027C0004B07209371073093720740937307509320
:1027D00074078091480790914907A0914A07B091EA
:1027E0004B072091C6013091C7010097A105B105A3
:1027F00011F4286001C0277F3093C7012093C601E0
:102800000895EF92FF920F931F93E0904807F09086
:10281000490700914A0710914B072091BD01309163
:10282000BE014091BF015091C0012E153F054007E8
:1028300051073CF48091C6019091C70184608C7F60
:102840000EC08091C6019091C701E216F3060407FD
:10285000150719F4897F816002C0887F8260909398
:10286000C7018093C6018091C6019091C701E11410
:10287000F1040105110511F4886001C0877F909370
:10288000C7018093C6011F910F91FF90EF900895AB
:1028900080913F07882339F48091C6019091C70148
:1028A00083FF7AC060C0813039F48091C601909175
:1028B000C70183FD71C057C0823029F48091C601E1
:1028C0009091C7012CC0833039F48091C60190915A
:1028D000C70180FD61C047C0843039F48091C601D2
:1028E0009091C70182FF58C03EC0853039F4809175
:1028F000C6019091C70182FD36C011C0863039F4FF
:102900008091C6019091C70181FF46C02CC08730DD
:1029100049F48091C6019091C70181FD24C080FFD8
:102920003BC021C0883039F48091C6019091C70125
:1029300084FF32C018C0893039F48091C60190916B
:10294000C70185FF29C00FC08A3039F48091C601C4
:102950009091C70186FF20C006C08B3069F480913A
:10296000C60187FF19C08091BB019091BC01909373
:102970003D0780933C0708958C3071F48091C60127
:102980009091C70190FF08C08091BB019091BC015C
:1029900090933D0780933C0708958091BB019091EF
:1029A000BC0190933D0780933C0708952091A701B7
:1029B0002830B8F4E22FF0E0EE0FFF1FE956FE4F8B
:1029C00080913C0790913D07918380832F5F2093F6
:1029D000A7018091BB019091BC0190933D0780932A
:1029E0003C070895E091A701EE2371F0E150E093D8
:1029F000A701F0E0EE0FFF1FE956FE4F80819181A5
:102A000090933D0780933C07089580913F07813064
:102A100011F480939601089580913F07813011F45D
:102A200010929601089510924707089580913F07EC
:102A3000882339F48091C6019091C7018F709070FE
:102A40001FC0813031F48091C6019091C7018F7E03
:102A500017C0823031F48091C6019091C7018F7DFB
:102A60000FC0833031F48091C6019091C7018F7BF4
:102A700007C0843051F48091C6019091C7018F77CF
:102A80009093C7018093C6010895853049F48091E1
:102A9000C6019091C7019E7F9093C7018093C601A4
:102AA000089580913F07813041F48091D30680934F
:102AB000E3018091D5068093E40108950895000014
:102AC0000895000008950000089500000895000092
:102AD0000895000008950000089500000895000082
:102AE0000895000008950000089500000895000072
:102AF0000895000008950000089500000895000062
:102B00000895000008950000089500000895000051
:102B10000895000008950000089500000895000041
:102B2000089510924707089580913F07813041F43E
:102B30008091BB019091BC0190933D0780933C072D
:102B400081E080934707089582E0809347070895C6
:102B500083E08093470710923D0710923C078FEF68
:102B60009FEF9093CB018093CA011092A70110921E
:102B70004C071092A80181E08093C3011092C90113
:102B80001092C801109248071092490710924A0704
:102B900010924B07109296010895109254071092CC
:102BA000C9011092C801089580913F078130D9F082
:102BB000813030F0823031F1833009F044C033C0CD
:102BC000809147078093D20680914C078093D1066D
:102BD0002091C8013091C901832F99278093D30692
:102BE0002093D5060895809147078093D20680915F
:102BF0004C078093D10680913D078093D306809146
:102C00003C070EC080914B078093D20680914A0703
:102C10008093D106809149078093D306809148071D
:102C20008093D5060895809174078093D206809191
:102C300073078093D106809172078093D3068091A9
:102C400071078093D50608958091D5068093610120
:102C500081E0809321078091E506882319F082E0C6
:102C60008093210780911C07882319F083E08093CB
:102C70002107089580916201882321F481E08093E7
:102C800062010895823019F483E08093620108950F
:102C900080913F07813049F08130A0F0823009F403
:102CA0004FC0833009F063C058C04091E10150919A
:102CB000E2016091BB017091BC01EDECF1E020E01C
:102CC00030E03AC02091E1013091E2012A30310533
:102CD00090F4F901EE0FFF1FE353FE4F8091BB010B
:102CE0009091BC01918380832F5F3F4F3093E2012D
:102CF0002093E101089589E080933B070895819135
:102D0000919186179707B1F4F901EE0FFF1FE35376
:102D1000FE4F4150504006C02F5F3F4F828193814C
:102D20008193919324173507B8F35093E2014093B0
:102D3000E10108952F5F3F4F2417350701F70895EC
:102D40001092E2011092E101EDECF1E0119211928A
:102D500081E0E13EF80771F0F9CF1092D2061092AF
:102D6000D1061092D3068AE08093D506089583E0B9
:102D700080933B07089580916A07813881F580919F
:102D80006B07823961F580916C07833A41F5809138
:102D90006D07843B21F580916E07853C01F580919C
:102DA0006F07863DE1F4F894C098AB9A89E0E3E0C0
:102DB000F0E0809357008491867019F40C940038E9
:102DC0000895823019F40C94003C0895843019F46D
:102DD0000C94003E0895863011F40C94003F089541
:102DE000CF93DF93CDB7DEB728970FB6F894DEBF49
:102DF0000FBECDBF80913F078130F1F48091400735
:102E00008A32C1F48091D50689838091D3068A8362
:102E10008091D1068B838091D2068C831D821E8285
:102E20001F821886BE016F5F7F4F8FEF97E00E9471
:102E30001D312FC084E02BC0882341F5BE016F5F98
:102E40007F4F8FEF97E00E94E7309091D506898100
:102E5000981799F49091D3068A81981771F49091FC
:102E6000D1068B81981749F49091D2068C819817DE
:102E700021F481E08093D50602C01092D50610920D
:102E8000D2061092D1061092D30603C083E080933D
:102E90003B0728960FB6F894DEBF0FBECDBFDF917B
:102EA000CF91089580914707882389F1833079F184
:102EB000853069F169EA71E080913C0790913D07A6
:102EC0000E94E73020913C0730913D078091CA0174
:102ED0009091CB018217930721F081E08093C30189
:102EE00002C01092C3013093CB012093CA012F5F1F
:102EF0003F4F30933D0720933C0780914707823036
:102F000019F485E08093470781E090E0089580E020
:102F100090E008958CE090E00E9411108093B2013F
:102F200080913F07882399F482E08093C40124E5CF
:102F300030E0A2EBB1E0F9018491FD0181832F5FC4
:102F40003F4F1196F1E0AA3BBF0761F0F4CF10921A
:102F5000D20681E08093D10683E08093D30685E298
:102F60008093D50608952091BB013091BC01309328
:102F7000C9012093C80182E08093C4012F5F3740CC
:102F800078F487E090E00E94111080FD09C063EBA7
:102F900071E08091C8019091C9010E94E73007C09B
:102FA000E2EBF1E0119281E0EB3BF807D9F78CE01E
:102FB00090E00E9411108093B201089583E0809305
:102FC000470787E090E00E94111081FD04C081E076
:102FD0008093540703C088E080933B078091BB0136
:102FE0009091BC019093C9018093C80108950F93FB
:102FF0001F93CF93DF93CDB7DEB724970FB6F89426
:10300000DEBF0FBECDBFE82FF0E06623C1F189E03F
:10301000689F800111249F0123703070C901880FBF
:10302000991F820F931F080F191F055E1D4F82E025
:103030000F3C180744F081E080933B0760E070E0AC
:1030400080E090E026C0C80102960E9411108B8398
:10305000C80101960E941110FE0131968183C801BA
:103060000E94111089838B8187FF03C08FEF8C83AF
:1030700001C01C8269817A818B819C810AC0EE0F1C
:10308000FF1FEE0FFF1FEB5AF84F608171818281A5
:10309000938124960FB6F894DEBF0FBECDBFDF91AB
:1030A000CF911F910F910895CF93DF93CDB7DEB7E6
:1030B00024970FB6F894DEBF0FBECDBF60913F07D7
:1030C000809140070E94F71769837A838B839C83E2
:1030D0004C814093D2063B813093D1062A812093C4
:1030E000D30699819093D506809161078823F9F0E2
:1030F00040934B0730934A07209349079093480722
:103100008091480790914907A0914A07B0914B07D9
:103110002091C6013091C7010097A105B10511F4B6
:10312000286001C0277F3093C7012093C6012496F1
:103130000FB6F894DEBF0FBECDBFDF91CF910895DB
:103140008091BB019091BC01825D944041F460E0AC
:1031500080E090E00E941910F8940C94000008950B
:103160000F931F93CF93DF93CDB7DEB724970FB69E
:10317000F894DEBF0FBECDBF90913F07992341F178
:1031800089E0989F800111248091400723E0829F6D
:10319000C0011124080F191F055E1D4F82E00F3C6E
:1031A000180724F081E080933B0732C06091D1067C
:1031B000C80102960E9419106091D306C8010196B9
:1031C0000E9419106091D506C8010E94191020C0F4
:1031D0008091D1068B839091D3069A839091D506E6
:1031E000998387FF03C08FEF8C8301C01C82E0911D
:1031F0004007F0E0EE0FFF1FEE0FFF1FEB5AF84FF6
:1032000089819A81AB81BC8180839183A283B383BE
:1032100024960FB6F894DEBF0FBECDBFDF91CF91DD
:103220001F910F91089590913F0797FF13C08091D0
:103230004B078093D20680914A078093D1068091F4
:1032400049078093D306809148078093D5069F77DE
:1032500090933F0790913F07992329F0923019F0FE
:10326000933009F046C0C39A8BB780648BBFC49A71
:103270008BB780648BBF992329F48BB78F7B8BBF6F
:10328000AF980DC0923029F48BB78F7B8BBFAE986F
:1032900006C0933021F48BB78F7B8BBFAD988091A4
:1032A0004007843030F08091D2060E94BB1080939A
:1032B000D20680914007833030F08091D1060E9481
:1032C000BB108093D10680914007823030F080910E
:1032D000D3060E94BB108093D3068091D5060E942E
:1032E000BB108093D50685B3806E85BB8BB7806499
:1032F0008BBF80913F07813051F585B3806E85BBD0
:103300008BB780648BBFC49A8BB780648BBF8BB73D
:103310008F7B8BBFC3988091D2060E94BB10809395
:10332000D2068091D1060E94BB108093D106809175
:10333000D3060E94BB108093D3068091D5060E94CD
:10334000BB108093D506C39A8BB780648BBF8091E6
:103350006107882359F18091D20680934B078091B1
:10336000D10680934A078091D306809349078091C4
:10337000D506809348078091480790914907A0910E
:103380004A07B0914B072091C6013091C7010097C1
:10339000A105B10531F428603093C7012093C6011F
:1033A0000895277F3093C7012093C60108951F9386
:1033B00081E080934C0740913F07442339F080918E
:1033C000BB019091BC011816190604F52091C301A8
:1033D000222341F08091BB019091BC019093C201E6
:1033E0008093C101442391F48091BB019091BC0171
:1033F0008F5F9F4F51F5222341F1809148079091B3
:1034000049079093C2018093C1011FC08091BB0105
:103410009091BC01181619061CF020E030E00AC09B
:1034200020E08091C1019091C201892B09F021E037
:1034300081E02827122F8091C6019091C701222395
:1034400011F0806121C08F7E1FC08091C1019091D9
:10345000C201892B11F410924C0780914C078823EC
:1034600041F08091CA019091CB0190933D078093E8
:103470003C078091C6019091C7018F7E9093C70150
:103480008093C60110E025C09093C7018093C601C8
:103490004130F9F460E08DE70E941C0890E0209133
:1034A0004007220F02C0959587952A95E2F780FF85
:1034B00002C010924C0780914C07882351F01123D1
:1034C00041F48091CA019091CB0190933D07809384
:1034D0003C0780913F07823019F563E08DE70E9439
:1034E0001C0890E040914007440F22E030E002C009
:1034F000220F331F4A95E2F782239323892B11F081
:1035000010924C0780914C07882351F0112341F40D
:103510008091CA019091CB0190933D0780933C0725
:1035200080913F078330F9F463E08DE70E941C0827
:1035300090E020914007220F02C0959587952A952B
:10354000E2F780FF02C010924C0780914C0788235D
:1035500051F0112341F48091CA019091CB019093D5
:103560003D0780933C0780913F07843009F049C0B4
:10357000E0914007E33050F410924C07F0E0EB503C
:10358000F94F8081882379F181E028C0E43049F443
:103590008091F506882301F520E030E08091F60661
:1035A00015C0E53059F0E63019F48091F50608C0F1
:1035B000E730B9F48091F506882371F48091F6061E
:1035C000882351F420E030E08091F706882311F041
:1035D00021E030E0C90102C081E090E080934C0717
:1035E00002C010924C0780914C07882351F01123A0
:1035F00041F48091CA019091CB0190933D07809353
:103600003C071F91089580913F07882341F4E09182
:103610004007F0E0EB50F94F81E08083089581305E
:1036200081F480914007E82FF0E0EB50F94F9FE0E4
:10363000908362E00E941509809140070E9467090B
:103640000895823049F5E0914007F0E0EB50F94FE2
:10365000E081E093D506809161078823E9F08E2F01
:1036600090E0A0E0B0E08093480790934907A093D2
:103670004A07B0934B078091C6019091C701EE2392
:1036800031F488609093C7018093C6010895877FC5
:103690009093C7018093C601089562E0809140072E
:1036A0000E941509809140070E9467090895EF92D2
:1036B000FF920F931F93CF93DF938091400788234E
:1036C00041F480913F07873109F001C10E94CD0983
:1036D000FEC0813009F0B0C080913F07863038F4D9
:1036E000C82FD0E0C759DE4F8330E1F415C08930D0
:1036F00038F4C82FD0E0CC0FDD1FCC59DE4F12C0FC
:103700008C3008F0E1C0C82FD0E0CC0FDD1FCC0F0B
:10371000DD1FCC5ADE4F06C0CE010E9411108093EF
:10372000D1050FC0843031F4CE010E941110809376
:10373000D00507C0853029F4CE010E941110809376
:10374000D20580913F07863061F4CE0101960E9438
:1037500011108093D405CE010E9411108093D305DF
:10376000B6C0873061F4CE0101960E94111080939B
:10377000CD05CE010E9411108093CC05A8C08830E1
:1037800061F4CE0101960E9411108093CF05CE0105
:103790000E9411108093CE059AC08930C1F4CE01E9
:1037A00003960E9411108093BA06CE0102960E94E1
:1037B00011108093B906CE0101960E9411108093DA
:1037C000B806CE010E9411108093B70680C08A30DF
:1037D000C1F4CE0103960E9411108093BE06CE0163
:1037E00002960E9411108093BD06CE0101960E94A0
:1037F00011108093BC06CE010E9411108093BB066D
:1038000066C08B3009F063C0CE0103960E94111090
:103810008093CB05CE0102960E9411108093CA05B9
:10382000CE0101960E9411108093C905CE010E941D
:1038300011108093C8054BC0823009F048C0009138
:103840003F07083308F043C010E0000F111F000FBE
:10385000111FBBE1EB2EB3E0FB2EE00EF11EC70102
:103860000E9411100A521A4FF801808380913F077D
:10387000C82FD0E0CC0FDD1FCC0FDD1FC952DA4FAF
:10388000C70101960E941110888380913F07C82FBD
:10389000D0E0CC0FDD1FCC0FDD1FC852DA4FC701BF
:1038A00002960E941110888380913F07C82FD0E0B4
:1038B000CC0FDD1FCC0FDD1FC752DA4FC7010396B7
:1038C0000E941110888303C0CFEFD3E02BCFDF918C
:1038D000CF911F910F91FF90EF9008950F931F9339
:1038E000CF93DF9380914007882321F480913F0795
:1038F000893449F089E090E00E941110882319F082
:1039000085E080933B0780914007882311F58091E3
:103910003F07803428F5873088F4863011F48EE72D
:103920000AC0880F880F8C590E94040B80913F07B2
:10393000880F880F8A590E94040BF0C0873019F451
:103940000E94C30AEBC0873109F0E8C00E94820AD6
:10395000E5C0813009F09FC080913F07833020F49B
:1039600083E080933B07DAC0863038F4C82FD0E07C
:10397000C759DE4F8330C9F415C0893038F4C82FD9
:10398000D0E0CC0FDD1FCC59DE4F0FC08C3008F0DB
:10399000C2C0C82FD0E0CC0FDD1FCC0FDD1FCC5A2A
:1039A000DE4F03C06091D10509C0843019F46091E5
:1039B000D00504C0853029F46091D205CE010E9463
:1039C000191080913F07863049F46091D405CE01EB
:1039D00001960E9419106091D3055BC0873049F4AD
:1039E0006091CD05CE0101960E9419106091CC0521
:1039F00050C0883049F46091CF05CE0101960E94F5
:103A000019106091CE0545C08930A9F46091BA06BD
:103A1000CE0103960E9419106091B906CE0102965C
:103A20000E9419106091B806CE0101960E941910EB
:103A30006091B7062EC08A30A9F46091BE06CE010F
:103A400003960E9419106091BD06CE0102960E9455
:103A500019106091BC06CE0101960E941910609168
:103A6000BB0617C08B3009F059C06091CB05CE0161
:103A700003960E9419106091CA05CE0102960E9419
:103A800019106091C905CE0101960E94191060912C
:103A9000C805CE013DC0823009F040C0E0913F072B
:103AA000E833E0F5F0E0EE0FFF1FEE0FFF1F8F0190
:103AB000055E1C4FEA52FA4F6381C80103960E94CB
:103AC0001910E0913F07F0E0EE0FFF1FEE0FFF1F10
:103AD000EA52FA4F6281C80102960E941910E091E1
:103AE0003F07F0E0EE0FFF1FEE0FFF1FEA52FA4F05
:103AF0006181C80101960E941910E0913F07F0E032
:103B0000EE0FFF1FEE0FFF1FEA52FA4F6081C80150
:103B10000E94191003C0CFEFD3E047CFDF91CF91C0
:103B20001F910F9108950F931F93CF93DF93CDB7FC
:103B3000DEB728970FB6F894DEBF0FBECDBF8091D9
:103B40004007882309F0DCC080913F0787FD7DC0D6
:103B5000803408F041C08630A9F48FE78093E106F5
:103B600066EE76E081EE96E00E94EF048091E90631
:103B70008093D5068091E8068093D3068091E7066E
:103B80008093D10680913F07873008F449C1880FA0
:103B9000880F8B598093E10666EE76E081EE96E021
:103BA0000E94EF048091E9068093D5068091E80693
:103BB0008093D3068091E1068E5F8093E10666EEE6
:103BC00076E081EE96E00E94EF048091E906809312
:103BD000D1068091E80636C0803519F486E090E081
:103BE00008C0813519F487E090E003C090E080546C
:103BF00090401092D3060E9411108093D5069091A8
:103C00003F07892F8654823008F00AC1963419F490
:103C10000EE411E002C00AE411E0C8010E94111094
:103C20008093D506C80101960E9411108093D30697
:103C3000C80102960E9411108093D106C801039614
:103C40000E9411108093D206EBC01092D2061092FF
:103C5000D1061092D306803819F48091470716C018
:103C6000813819F48091540711C0823859F4809139
:103C70003C0790913D07892F99278093D306809127
:103C80003C0704C0833829F48091A8018093D506AD
:103C90002FC08438C9F4F8948091F1069091F2060F
:103CA000A091F306B091F40689839A83AB83BC8319
:103CB000789489818093D5068A818093D3068B81FD
:103CC0008093D1068C8112C0853891F40E94623CA9
:103CD0006D837E838F8398878D818093D5068E81B7
:103CE0008093D3068F818093D10688858093D206F6
:103CF00080913F078F3F09F093C08091C5018EC02E
:103D0000813009F074C01092D2061092D106109240
:103D1000D30680913F07882319F48091D50515C0FB
:103D20008130A9F0823019F48091B6060EC083303C
:103D300019F48091D10509C0843019F48091D0051F
:103D400004C0853021F48091D2058093D5068091FE
:103D50003F07863039F48091D4058093D306809153
:103D6000D3055CC0873039F48091CD058093D306AC
:103D70008091CC0553C0883039F48091CF05809371
:103D8000D3068091CE054AC0893079F48091BA0675
:103D90008093D2068091B9068093D1068091B806AF
:103DA0008093D3068091B70639C08A3079F4809128
:103DB000BE068093D2068091BD068093D106809185
:103DC000BC068093D3068091BB0628C08B3041F59A
:103DD0008091CB058093D2068091CA058093D1064D
:103DE0008091C9058093D3068091C80517C08230A1
:103DF000B9F4E0913F07E83398F4F0E0EE0FFF1FCD
:103E0000EE0FFF1FEA52FA4F83818093D206828120
:103E10008093D10681818093D30680818093D506DB
:103E200080916107882339F18091D20680934B07F6
:103E30008091D10680934A078091D30680934907E9
:103E40008091D50680934807809148079091490753
:103E5000A0914A07B0914B072091C6013091C7014C
:103E60000097A105B10511F4286001C0277F3093A8
:103E7000C7012093C60128960FB6F894DEBF0FBE87
:103E8000CDBFDF91CF911F910F910895EF92FF92D7
:103E90000F931F93CF93DF9380914007882309F0FE
:103EA00024C180913F0787FDEEC0803458F58630ED
:103EB00061F42091D506207F6091D1066F7C60620D
:103EC0004091D3068EE70E94E90500913F07073035
:103ED00008F4BBC110E0000F111F000F111F20914B
:103EE000D5064091D30660E0802F8C590E94E905E9
:103EF0002091D1064091D20660E0802F8A590E941D
:103F0000E905A3C1893409F58091BB019091BC01F9
:103F100024E0823D920731F41092D30681E0809331
:103F2000D5060CC0815E904129F41092D306109200
:103F3000D50604C084E080933B0787C16091D50615
:103F400089E090E00E94191080C1803519F4C6E024
:103F5000D0E015C0813529F0C82FD0E0C054D04042
:103F60000EC08091D50680FD08C087E090E00E94D9
:103F7000111080FF02C00E946B30C7E0D0E080913A
:103F80003F07873419F4CAE4D1E004C0863411F441
:103F9000CEE4D1E08654823090F46091D206CE0116
:103FA00003960E9419106091D106CE0102960E94DC
:103FB00019106091D306CE0101960E9419106091EC
:103FC000D506CE010E94191080913F07873411F069
:103FD000853449F58AE491E00E94111080933507F9
:103FE0008BE491E00E941110809336078CE491E0FD
:103FF0000E941110809337078DE491E00E94111008
:1040000080933807E0903507F09036070091370726
:104010001091380785E090E00E941110B801A701C7
:1040200090E00E94B63480913F078634C1F48EE45C
:1040300091E00E9411108093ED068FE491E00E94C0
:1040400011108093EE0680E591E00E94111080939C
:10405000EF0681E591E00E9411108093F0068091B7
:104060003F07823421F48091D5060E944B3780911E
:104070003F07833409F0E9C08091D50682958F709F
:1040800080936301E2C0833829F48091D506809340
:10409000A80121C0843899F4F8948091BD019091D1
:1040A000BE01A091BF01B091C0018093F106909331
:1040B000F206A093F306B093F40678940CC085380A
:1040C00051F46091BD017091BE018091BF0190914A
:1040D000C0010E94673C80913F078F3F09F0B5C047
:1040E0008091D5068093C501B0C0813009F094C09D
:1040F00080913F07882329F48091D5068093D505C8
:10410000A4C0813009F44FC0823029F48091D506D3
:104110008093B6069AC0833029F48091D5068093A7
:10412000D10593C0843029F48091D5068093D005C1
:104130008CC0853029F48091D5068093D20585C046
:10414000863079F48091D30690E0982F88272091CB
:10415000D50630E0822B932B9093D4058093D30522
:1041600074C0873079F48091D30690E0982F882727
:104170002091D50630E0822B932B9093CD05809330
:10418000CC0563C0883079F48091D30690E0982FF5
:1041900088272091D50630E0822B932B9093CF0572
:1041A0008093CE0552C0893089F48091BD019091F1
:1041B000BE01A091BF01B091C0018093B70690935A
:1041C000B806A093B906B093BA063FC08A3089F406
:1041D0008091BD019091BE01A091BF01B091C0013D
:1041E0008093BB069093BC06A093BD06B093BE0619
:1041F0002CC08B3051F58091BD019091BE01A091F2
:10420000BF01B091C0018093C8059093C905A093E8
:10421000CA05B093CB0519C08230B9F4E0913F07CD
:10422000E83398F4F0E0EE0FFF1FEE0FFF1FEA52A5
:10423000FA4F8091D20683838091D1068283809148
:10424000D30681838091D5068083DF91CF911F9122
:104250000F91FF90EF90089530914B073093D20665
:1042600020914A072093D106909149079093D30655
:10427000809148078093D5069093BC018093BB0141
:104280003093C0012093BF019093BE018093BD0184
:104290000E94461F08950F931F93CF93DF93E091E1
:1042A0003F07E7FD08C0EF3008F0B9C0F0E0E05983
:1042B000FE4FE49101C0EF77E0933F0790913F07F5
:1042C0009034C8F4E92FF0E0009140079F3040F4AB
:1042D000EE0FFF1F0295000F007E802F8E2B08C06F
:1042E000EB5AFE4F8491880F0295000F007E802BC1
:1042F0000E944E0B94C09B34E1F480914007C82F7C
:10430000D0E0CC0FDD1FCE01865A9E4F0E941110C7
:10431000CA5ED84F888380914007C82FD0E0CC0F69
:10432000DD1FCE01855A9E4F0E941110CA5ED84FE4
:104330001DC09C34E9F480914007C82FD0E0CC0F19
:10434000DD1FCE01805A9E4F0E941110C850D94FD8
:10435000888380914007C82FD0E0CC0FDD1FCE01AD
:104360008F599E4F0E941110C850D94F898357C052
:104370009335E1F480914007C82FD0E0CC0FDD1FCA
:10438000CE018A599E4F0E941110C55ADE4F888374
:1043900080914007C82FD0E0CC0FDD1FCE01895996
:1043A0009E4F0E941110C55ADE4FE0CF892F8155D4
:1043B000823020F483E080933B0731C000914007B6
:1043C0009D3459F410E0C80183509C4F0E94111095
:1043D000035E184FF801808322C0C02FD0E0C05C7C
:1043E000D04083E0989FC0011124C80FD91FCE018F
:1043F00040960E9411108093D506682F8C2F0E9442
:104400009F1080913F07853451F4CE010D960E9494
:104410001110682F9E012350822F0E949F10DF9160
:10442000CF911F910F9108951F93CF93DF93E09148
:104430003F07E7FD08C0EF3008F0B3C0F0E0E059F7
:10444000FE4FE49101C0EF77E0933F0720913F07D3
:104450002034D0F4E22FF0E0909140072F3040F468
:10446000EE0FFF1F9295990F907E892F8E2B08C01B
:10447000EB5AFE4F8491880F9295990F907E892B6D
:104480000E94040B182F88C02B34C9F48091400778
:1044900090E0880F991FFC01EA5EF84F6081865A10
:1044A0009E4F0E9419108091400790E0880F991F3D
:1044B000FC01EA5EF84F6181855A9E4F1AC02C3488
:1044C000D9F48091400790E0880F991FFC01E850D3
:1044D000F94F6081805A9E4F0E94191080914007C9
:1044E00090E0880F991FFC01E850F94F61818F59C6
:1044F0009E4F0E94191055C02335C9F48091400782
:1045000090E0880F991FFC01E55AFE4F60818A599F
:104510009E4F0E9419108091400790E0880F991FCC
:10452000FC01E55AFE4F618189599E4FE2CF2D343F
:1045300051F48091400790E0FC01E35EF84F608108
:1045400083509C4FD6CF822F8155823010F483E068
:1045500026C080914007C82FD0E0C05CD04083E0E7
:10456000289FC0011124C80FD91F8C2F0E949810BA
:10457000682FCE0140960E941910182F80913F0796
:10458000853451F49E012350822F0E949810682F89
:10459000CE010D960E941910123019F485E0809317
:1045A0003B07DF91CF911F910895DF92EF92FF9229
:1045B0000F931F93CF93DF93CDB7DEB726970FB638
:1045C000F894DEBF0FBECDBFE0913F07E7FD08C006
:1045D000EF3008F00FC2F0E0E059FE4FE49101C067
:1045E000EF77E0933F0720913F072B3108F0B3C0EE
:1045F000233041F4E0914007F0E0EE0FFF1FED594A
:10460000F84F09C0263061F4E0914007F0E0EE0F6A
:10461000FF1FE35BF84F81818093D306808190C0B8
:1046200090914007E22FF0E0293058F5EE0FFF1F80
:104630009295990F907E9E2B91609093E10666EE85
:1046400076E081EE96E00E94EF048091E706809389
:10465000D1069091E8069093D3068091E906809365
:10466000D50680913F07843008F46CC093FF6AC080
:10467000906F9093D3068FEF8093D1068093D206EC
:1046800061C0EB5AFE4F8491880F9295990F907EEE
:10469000982B91609093E10666EE76E081EE96E0CD
:1046A0000E94EF041E828091E7068D838091E806C8
:1046B0008C838091E9068B832B813C814D815E81C7
:1046C000E0913F078E2F90E0FC01ED5BFE4FE491FF
:1046D00004C05595479537952795EA95D2F72B83D2
:1046E0003C834D835E83815D9E4FEE24FF248701D2
:1046F00060E070E0FC01D4900FC081E090E0A0E0A9
:10470000B0E004C0880F991FAA1FBB1FEA95D2F71B
:10471000E82AF92A0A2B1B2BE62F6F5F7F4FED1536
:1047200060F3E222F32204231523EB82FC820D8343
:104730001E838D818093D1068C818093D3068B81DB
:104740008093D5068091D10687FF02C08FEF25C1E7
:104750001092D20624C12E3108F03FC01092D2062A
:104760001092D1061092D3061092D5068DE7809351
:10477000E10666EE76E081EE96E00E94EF0480911D
:104780003F078B3199F480914007880F22E030E099
:1047900002C0220F331F8A95E2F78091E90690E06C
:1047A00028233923232B09F4FAC015C08C3119F4BE
:1047B0008091E90605C08D3109F0F1C08091E606CF
:1047C00090E020914007220F02C0959587952A9589
:1047D000E2F780FFE4C081E0A0C0203408F4DFC02D
:1047E000203608F09DC010914007105C83E0289FA0
:1047F000C0011124180F253431F4812F83500E94F9
:1048000098108093D306812F0E9498108093D5062C
:1048100080913F078B34A9F4E0914007F0E0EE0F60
:10482000FF1FEA5EF84F91819093D30680818093B9
:10483000D50697FF27C08FEF8093D2068093D106CD
:1048400021C08C3441F4E0914007F0E0EE0FFF1FEF
:10485000E850F94F09C0833559F4E0914007F0E082
:10486000EE0FFF1FE55AFE4F81818093D30607C0EC
:10487000863541F4E0914007F0E0E05AFF4F808137
:104880008093D50680913F078D3431F4E091400745
:10489000F0E0E35EF84F0FC08E3431F4E091400752
:1048A000F0E0E651F94F07C0803541F4E091400750
:1048B000F0E0ED5FF84F80818093D50680913F074F
:1048C0008135A1F4809140070E94ED386B837C8391
:1048D0008D839E838E818093D2068D818093D106B5
:1048E0008C818093D3068B818093D50680913F077E
:1048F000873419F0803409F052C09091D50684E6CF
:10490000989FC001112461E170E00E94E63C7A8327
:1049100069838A818093D30689818093D5063FC0BD
:104920002236C1F41092D306E0914007F0E0EC5B30
:10493000F84F808181FF04C081E08093D50602C0DA
:104940001092D506E0914007F0E0EC5BF84F8081D3
:104950008D7F808380913F078336C1F41092D30608
:10496000E0914007F0E0EC5BF84F808182FF04C0EB
:1049700081E08093D50602C01092D506E0914007F1
:10498000F0E0EC5BF84F80818B7F80838091D306D1
:1049900087FF05C08FEF8093D1068093D206809168
:1049A0006107882339F18091D20680934B0780916B
:1049B000D10680934A078091D3068093490780915E
:1049C000D506809348078091480790914907A091A8
:1049D0004A07B0914B072091C6013091C70100975B
:1049E000A105B10511F4286001C0277F3093C701EC
:1049F0002093C60126960FB6F894DEBF0FBECDBF3A
:104A0000DF91CF911F910F91FF90EF90DF9008956C
:104A10000F931F93CF93DF93982FC82FDD27C7FDE8
:104A2000D095FE01EF5BF84F8081882319F480E078
:104A300090E01EC010828E01000F111FF801E35B91
:104A4000F84F60817181892F0E9489080D59184F94
:104A500025E0CC0FDD1F2A95E1F7F8012081418187
:104A600060E0FE01E6608E2F0E94E90581E090E0A3
:104A7000DF91CF911F910F910895CF93DF93CDB721
:104A8000DEB722970FB6F894DEBF0FBECDBF909170
:104A90004007E92FF0E0EF5BF84F8081813019F497
:104AA000892F0E9408258091BB019091BC019095AF
:104AB00081959F4F9A83898362E0809140070E948D
:104AC0001509809140078295880F807E29814A814F
:104AD00060E088600E94E905809140078295880F18
:104AE000807E2FEF47E060E086600E94E905E0915C
:104AF0004007F0E0EF5BF84F82E0808322960FB62C
:104B0000F894DEBF0FBECDBFDF91CF910895909195
:104B10004007E92FF0E0EF5BF84F8081813019F416
:104B2000892F0E94082562E0809140070E941509A4
:104B3000809140078295880F807E2091D506409114
:104B4000D30660E088600E94E90580914007829565
:104B5000880F807E2FEF47E060E086600E94E905C5
:104B6000E0914007F0E0EF5BF84F82E0808308952A
:104B7000DF92EF92FF920F931F93CF93DF93CDB706
:104B8000DEB724970FB6F894DEBF0FBECDBFD62E8A
:104B9000082F10E0C801E5E0880F991FEA95E1F7BA
:104BA00082600E945A089B01AC01DD2069F1780106
:104BB000EE0CFF1CE00EF11E8BE192E0E80EF91EF8
:104BC00089E0D89EC0011124E80EF91E9FECE91679
:104BD00092E0F90624F081E080933B0720C029830E
:104BE0003A834B835C836B81C70102960E94191044
:104BF000FE0131966181C70101960E9419106981F9
:104C0000C7010E9419100BC0000F111F000F111FC8
:104C10000B5A184FF8012083318342835383249623
:104C20000FB6F894DEBF0FBECDBFDF91CF911F91BD
:104C30000F91FF90EF90DF9008951F9310913F0721
:104C400080914007833010F4612F30C0843041F4EC
:104C5000612F80E00E94B825612F81E00E94B82575
:104C600080914007853041F4612F81E00E94B82592
:104C7000612F82E00E94B82580914007863041F480
:104C8000612F80E00E94B825612F82E00E94B82544
:104C900080914007873061F4612F80E00E94B82541
:104CA000612F81E00E94B825612F82E00E94B82523
:104CB0001F910895CF92DF92EF92FF920F931F936F
:104CC000182F062F8295880F807E82600E945A08D6
:104CD0006B017C01602F812F0E94F7176C157D05F9
:104CE0008E059F0529F460E070E080E090E010C040
:104CF000C616D706E806F9062CF46C197D098E094C
:104D00009F0906C0C61AD70AE80AF90AC701B60100
:104D10001F910F91FF90EF90DF90CF9008950F9328
:104D20001F93182F062F60E00E941509602F812F16
:104D30000E94F717AB01BC01812F8295880F807EFE
:104D40000E9431091F910F9108954F925F926F92C7
:104D50007F928F929F92AF92BF92CF92DF92EF920B
:104D6000FF920F931F93CF93DF93CDB7DEB72897B2
:104D70000FB6F894DEBF0FBECDBF4091D206488774
:104D80002091D1062F833091D3063E838091D506A2
:104D90008D83E0913F07E7FD08C0EF3008F09EC12A
:104DA000F0E0E059FE4FE49101C0EF77E0933F0758
:104DB000E0913F07E73411F0E03479F48091BB01D2
:104DC0009091BC0153E0880F991F5A95E1F76FE26B
:104DD00070E00E94FA3C6093D506E03408F0E8C029
:104DE000E930B0F5E63081F46091BB017091BC010F
:104DF000809140070E948908E0914007F0E0EE0FA3
:104E0000FF1FE35BF84FDDC02093E2063093E3061B
:104E10008091D5068093E406EE0F8091400782953D
:104E2000880F807E8E2B8093E10666EE76E081EE21
:104E300096E00E94EF0480913F07833009F042C161
:104E4000E0914007F0E0EE0FFF1FED59F84FB9C0B9
:104E5000E031E9F4809140078295880F807E81617E
:104E60008093E10666EE76E081EE96E00E94EF0424
:104E7000809140078295880F807E80618093E10653
:104E80009091D5069F708091E706807F1FC090911A
:104E90004007E13169F59295990F907E9161909369
:104EA000E10666EE76E081EE96E00E94EF048091E6
:104EB00040078295880F807E80618093E106909103
:104EC000D5069295907F8091E7068F70982B9093EE
:104ED000E2068091E8068093E3068091E9068093DC
:104EE000E40666EE76E081EE96E00E94EF04EAC00A
:104EF0001C822B833A838091D5068983F0E0EB5A9C
:104F0000FE4FE491EE0FB92EB294BB0C90EEB92295
:104F1000BE2A8B2D0E945A08AB01BC01E0913F07CD
:104F20008E2F90E0FC01ED5BFE4FE49101E010E07C
:104F300020E030E004C0000F111F221F331FEA954C
:104F4000D2F7C980DA80EB80FC8044245524815D4F
:104F50009E4FFC01A49025C03601470104C09594E2
:104F60008794779467948A95D2F7D401C3018170AE
:104F70009070892B29F0402B512B622B732B0AC088
:104F8000D901C80180959095A095B09548235923E3
:104F90006A237B23000F111F221F331F0894411C1B
:104FA000511C842D4A14C0F28B2D0E9431098AC0F5
:104FB000EB3471F4E0914007F0E0EE0FFF1FEA5E82
:104FC000F84F8091BB019091BC01918380837AC09E
:104FD000EC3441F4E0914007F0E0EE0FFF1FE850A1
:104FE000F94FEFCFE33541F4E0914007F0E0EE0FE9
:104FF000FF1FE55AFE4FE5CFE63531F4E09140075B
:10500000F0E0E05AFF4F07C0ED3449F4E09140076B
:10501000F0E0E35EF84F8091D506808353C0E13520
:1050200079F44C832B833A838091D5068983498117
:105030005A816B817C81809140070E942A3842C04E
:10504000E235C1F44C832B833A838091D506898362
:1050500069817A818B819C81462F4F71F5E095950E
:10506000879577956795FA95D1F7809140070E94CB
:10507000503828C0E03630F510914007105C83E0CE
:10508000E89FC0011124180FE53429F4632F812F04
:1050900083500E949F106091D506812F0E949F101F
:1050A000809140078B5E0E949810682F8091400786
:1050B0000E94E00F80913F07873411F0803411F493
:1050C0001092D30688858093D2068F818093D10673
:1050D0008E818093D3068D818093D50628960FB656
:1050E000F894DEBF0FBECDBFDF91CF911F910F911E
:1050F000FF90EF90DF90CF90BF90AF909F908F90F8
:105100007F906F905F904F90089530914B07309350
:10511000D20620914A072093D10690914907909397
:10512000D306809148078093D5069093BC01809365
:10513000BB013093C0012093BF019093BE018093C7
:10514000BD010E94A52608951092D2061092D106A4
:105150001092D30680914007882331F580913F0754
:10516000883018F40E94AB0F1DC08A30A0F40E9452
:10517000DD0F90E020913F0730E02850304002C022
:10518000959587952A95E2F780FF02C081E00AC0D5
:105190001092D50609C083B390E0969587959695B1
:1051A000879581708093D50680914007813081F486
:1051B000E0913F07F0E0EE0FFF1FEA5FF84F20811C
:1051C0003181818183708093D3062093D50608C0F6
:1051D000823031F480913F070E94CF0F8093D50633
:1051E00080916107882359F18091D20680934B0703
:1051F0008091D10680934A078091D3068093490716
:105200008091D5068093480780914807909149077F
:10521000A0914A07B0914B072091C6013091C70178
:105220000097A105B10531F428603093C7012093A0
:10523000C6010895277F3093C7012093C6010895C2
:1052400080914007882339F46091D50680913F070B
:105250000E94B50F0895823071F48091D50680FFC9
:1052600005C080913F070E94A30F089580913F07DA
:105270000E94A70F08958F3F21F56091D50680E029
:105280000E9450056091D30681E00E945005609114
:10529000D10682E00E9450058091D50682FF03C0AE
:1052A00080E00E9467098091D30682FF03C081E0FD
:1052B0000E9467098091D10682FF03C082E00E94AC
:1052C000670908950F931F93CF93DF93CDB7DEB790
:1052D0002F970FB6F894DEBF0FBECDBF8091440765
:1052E0009091BF06892B8093440780914507909148
:1052F000C006892B809345078091C106909146078F
:10530000892B8093460780912007882349F080915C
:10531000C6019091C70191609093C7018093C60127
:105320008091390780FF0BC08091C1019091C2012B
:10533000009729F001979093C2018093C1010E94C8
:105340000E0A282F8093EF014091ED015091EE015C
:105350004130510519F0882309F4A1C03091E506C8
:10536000832F8150823010F02230E1F58091ED06DC
:105370009091EE06A091EF06B091F0068C839D838C
:10538000AE83BF831A821B822230C1F0313011F408
:1053900097E001C098E0E3EBF1E0DE01189681911F
:1053A0008D9321E0EB3BF207D1F79983CE01019673
:1053B0000E947D35882309F47DC222C0E4E2F7E033
:1053C000DE01189681918D9387E0EC32F807D1F7D2
:1053D00087E08983CE0101960E947D35882309F4F8
:1053E00069C25AC080911C07882319F4233091F4B4
:1053F0000DC0233059F068E083EB91E00E947537CF
:105400008091ED019091EE018E7F50C268E084E2C0
:1054100097E0F4CF8091FE06882309F04BC280917B
:105420006201213039F14E7F5093EE014093ED013E
:105430008230A0F402EB11E0F80181918F010E940B
:105440001030F1E00B3B1F07B9F78091620181300A
:1054500009F030C282E0809362012CC282EB91E0BD
:105460000E94813980916201833009F023C2109239
:10547000620120C2882361F403E217E0F801819100
:105480008F010E941030F7E00C321F0729F0F6CF91
:1054900082EB91E00E9481391092EF010BC21092D1
:1054A000CC0180916201882331F489E697E00E9463
:1054B0003507813051F0809162018823A1F189E69E
:1054C00097E00E94173A813071F581E08093CC011A
:1054D000809169078093750780916A0780933F07E1
:1054E00080916B078093400780916C078093D20670
:1054F00080916D078093D10680916E078093D306CB
:1055000080916F078093D50680914707882319F40F
:1055100081E090E053C020E030E0833011F421E0DE
:1055200030E0C9014BC08091390782FF23C08091D0
:105530004707813009F044C090919601913009F0FD
:105540003FC083E08093CC0187E180937507109280
:105550003F07109240071092D2061092D106809118
:10556000E3018093D3068091E4018093D506909364
:10557000610726C00E945217882311F182E08093B0
:10558000CC018091A901809375078091AA01809335
:105590003F078091AB01809340078091AC018093DD
:1055A000D2068091AD018093D1068091AE018093A7
:1055B000D3068091AF018093D50681E08093610787
:1055C0008091CC01882309F475C182E090E00E94AB
:1055D0001110382F809353072091D3062093BC01DC
:1055E0009091D5069093BB018091D2068093C00123
:1055F0008091D1068093BF012093BE019093BD019D
:1056000010923B0790917507892F8854883310F0CA
:105610009E3870F08091CC01813011F4923F41F0BE
:1056200082E080933B078091A80181608093A8016C
:105630008091CC01813091F4E9E6F7E08191380F57
:1056400027E0E037F207D1F73093530780917007D6
:105650003817C9F081E080933B0715C0823099F478
:10566000E9EAF1E08191380F81E0E03BF807D1F7FA
:10567000309353078091B001381729F08091A80129
:1056800082608093A8011092C40180913B07882317
:1056900009F095C080915407882311F097FF50C0FE
:1056A000923F21F40E94BB1682E087C0E92FF0E010
:1056B00097FF05C0EE0FFF1FED50F04004C0EE0F46
:1056C000FF1FED59FF4F0190F081E02D84E680939C
:1056D0003B078091F001882311F0099503C08FEFFB
:1056E00080933B076091E1017091E20161157105C2
:1056F00009F465C080914707813009F060C080914E
:10570000CC01823009F05BC040913C0750913D07CD
:1057100020E030E00FC02F5F3F4FEE0FFF1FE3533D
:10572000FE4F808191814817590721F485E08093CD
:10573000470745C0E22FF0E0E617F70760F33FC0E8
:105740008091C8019091C901E7E08F3F9E07A0F5C5
:1057500069E677E00E941D31882371F565EE71E0FE
:105760008091C8019091C9010E94E73085E680933D
:105770003B0720E030E0F901EB51FE4FD901A7597A
:10578000B84F90818C91981721F087E080933B0768
:1057900005C02F5F3F4F2830310569F780913B07E7
:1057A000853669F48091C8019091C9010196909362
:1057B000C9018093C80103C087E080933B078091B3
:1057C000CC01813009F076C08CE090E00E9411108D
:1057D000182F82E090E00E941110282F80933E073E
:1057E0008091C4018823C9F590917507963031F4F2
:1057F0008091D106880F880B8093D2061093B20156
:105800002093B30180913B078093B4019093B5013D
:105810008091D2068093B6018091D1068093B70122
:105820008091D3068093B8018091D5068093B90109
:1058300080911C07882339F01092530790915307E9
:10584000E3EBF1E003C010935307F8CF8191980F79
:1058500021E0EA3BF207D1F70FC0813089F41093C1
:10586000B20110925307E2EBF1E090E08191980FC2
:1058700081E0EA3BF807D1F7909353079093BA0180
:105880008BE090E00E9411108093FE068091C5018C
:10589000882351F080917507863031F08A3021F0ED
:1058A0008F3011F08F3131F481E090E09093EE0170
:1058B0008093ED012F960FB6F894DEBF0FBECDBFDB
:1058C000DF91CF911F910F9108959F92AF92BF9258
:1058D000CF92DF92EF92FF920F931F93CF93DF93BC
:1058E000CDB7DEB722970FB6F894DEBF0FBECDBF9F
:1058F0006C017B01042F6115710509F499C00097B3
:1059000009F496C06817790709F492C0142F12950C
:10591000110F107EA6E09A2E912A892D0E94400830
:105920009A838983812F8C600E9440085C0180E00B
:10593000D7FC07C0EE0CFF1CCC0CDD1C8F5F8F303A
:10594000B9F7E114F10419F471E0E72EF12C40E00D
:1059500050E001C07901142F4F5F5F4FC701807085
:105960009E7F970136952795892BA1F7C9018C0D4C
:105970009D1DB7010E94E63CFB01672B11F4E1E09D
:10598000F0E089819A8154E0880F991F5A95E1F7D8
:10599000BF010E94E63C9B01C50144E0880F991FAE
:1059A0004A95E1F7BF010E94E63C412F50E01530D7
:1059B00090F484E090E0841B950B082E02C036958D
:1059C00027950A94E2F73A83298302C07695679572
:1059D0008A95E2F70FC0CA010497082E02C0220F71
:1059E000331F0A94E2F73A83298302C0660F771FB8
:1059F0008A95E2F789819A81892B21F481E090E0F0
:105A00009A8389836115710511F461E070E07497E0
:105A100018F4802F0E94890829814A8160E0892D2D
:105A20000E94E905E02FF0E0EF5BF84F81E0808312
:105A300022960FB6F894DEBF0FBECDBFDF91CF9197
:105A40001F910F91FF90EF90DF90CF90BF90AF909C
:105A50009F9008950F931F93CF93DF93CDB7DEB739
:105A600062970FB6F894DEBF0FBECDBF082F162F7A
:105A70008430C1F480E00E94082581E00E9408255E
:105A8000612F80E00E945A266F83788789879A87E2
:105A9000612F81E00E945A266B877C878D879E87C5
:105AA000198A3FC0853041F481E00E94082582E0D8
:105AB0000E940825198625C0863081F480E00E9466
:105AC000082582E00E940825612F80E00E945A2666
:105AD0006F83788789879A871D861BC0873009F571
:105AE00080E00E94082581E00E94082582E00E9453
:105AF0000825612F80E00E945A266F837887898766
:105B00009A87612F81E00E945A266B877C878D8758
:105B10009E87612F82E00E945A266F87788B898B3F
:105B20009A8B9985992331F48D85882319F4898975
:105B3000882369F09A83FE013796818189838D8558
:105B40008C838C858B8389898E8388890BC088851B
:105B50008A838F8189838C858C838B858B838889CD
:105B60008E838F858D83043049F429813A818B811E
:105B70009C8182179307D0F441E015C0053049F4A9
:105B80002B813C818D819E818217930758F041E0E3
:105B90000EC0063071F429813A818D819E81821771
:105BA000930720F442E0BC01C90133C040E0B901D1
:105BB00030C0073081F589819A812B813C81ED814C
:105BC000FE812817390768F4E817F907C0F441E0A7
:105BD000B9010E94652C6D817E8142E089819A81A4
:105BE00018C0E217F30758F440E0BC01C9010E9455
:105BF000652C6D817E8142E08B819C810AC040E0F2
:105C0000BC01CF010E94652C6B817C8141E08D81BC
:105C10009E810E94652C62960FB6F894DEBF0FBE7F
:105C2000CDBFDF91CF911F910F910895CF92DF9259
:105C3000EF92FF920F931F93CF93DF93CDB7DEB711
:105C400024970FB6F894DEBF0FBECDBF80913F07FB
:105C5000823008F04BC060E0809140070E94150937
:105C6000809140070E9408256E010894C11CD11C38
:105C70008091D2068C838091D1068B838091D3064C
:105C8000F60181838091D506898380913F07813019
:105C900009F5E980FA800B811C818091400782958B
:105CA000880F807E82600E945A08E60EF71E081F49
:105CB000191FE982FA820B831C838C818093D206A0
:105CC0008B818093D106F60181818093D3068981EF
:105CD0008093D50649815A816B817C8180914007F0
:105CE0008295880F807E0E94310946C0823009F07B
:105CF00043C0E090D50680914007833030F40E9485
:105D000008256E2D8091400735C06E2D0E942A2DEA
:105D100080914007843041F46E2D80E00E948F26F0
:105D20006E2D81E00E948F2680914007853041F4DE
:105D30006E2D81E00E948F266E2D82E00E948F26BC
:105D400080914007863041F46E2D80E00E948F26BE
:105D50006E2D82E00E948F2680914007873061F48B
:105D60006E2D80E00E948F266E2D81E00E948F268E
:105D70006E2D82E00E948F2624960FB6F894DEBF27
:105D80000FBECDBFDF91CF911F910F91FF90EF908C
:105D9000DF90CF900895CF92DF92EF92FF920F9312
:105DA0001F93CF93DF9310923D0710923C078FEF24
:105DB0009FEF9093CB018093CA018DE090E00E9409
:105DC0001110813011F4809347071DE4C12E17E0B4
:105DD000D12EB3E6EB2EB7E0FB2EC0E0D0E0CE0133
:105DE0008295880F807E182F8C600E944008F601F3
:105DF000819391936F01812F86600E944008F70183
:105E0000819391937F012196C330D10541F706ED2F
:105E100015E0CEE1D3E0CE010E941110F80183839A
:105E2000CE0101970E941110F8018283CE010297E2
:105E30000E941110F8018183CE0103970E94111076
:105E4000F801808324960C5F1F4FF3E0CE3FDF07FD
:105E500011F7ECEFFFE7E491E73299F4EDEFFFE79C
:105E6000E491E83171F4EEEFFFE7E491E83249F4B0
:105E7000EFEFFFE7E491E83121F481E08093F00156
:105E800002C01092F001DF91CF911F910F91FF900E
:105E9000EF90DF90CF9008951F920F920FB60F9260
:105EA00011248F939F93EF93FF938BB1887129F007
:105EB0008091F10180628093F101869B04C08CB1D6
:105EC000809323021AC080910D029CB1E82FF0E06C
:105ED000EE50FE4F90838F5F80930D028B3110F058
:105EE00010920D0290910D0280910E02981729F4E4
:105EF0008091F10180688093F101FF91EF919F9172
:105F00008F910F900FBE0F901F9018951F920F92B8
:105F10000FB60F9211248F939F93EF93FF9390915D
:105F2000220280912102981781F0969AE92FF0E0E1
:105F3000E15FFD4F80818CB9892F8F5F80932202B2
:105F4000823120F01092220201C05598FF91EF910A
:105F50009F918F910F900FBE0F901F9018951F92D9
:105F60000F920FB60F9211248F939F93909122025C
:105F700080912102981709F496989F918F910F9024
:105F80000FBE0F901F901895982F80910D0280934F
:105F90000E0280912202809321021092F101209141
:105FA000DA06283019F4EEE7F1E002C0E7E8F1E0A4
:105FB000849189B988ED8AB9992369F0993058F4A8
:105FC000E92FF0E0283019F4E258FE4F02C0E957FB
:105FD000FE4F849189B908958091F10181FF02C03B
:105FE0001092F1018BB1887129F08091F1018062EA
:105FF0008093F1018091F10182608093F101807FB3
:1060000019F08FEF9FEF089520E030E090910E029D
:1060100080910D02981711F021E030E0C901089538
:10602000969A90912102E92FF0E0E15FFD4F808385
:106030009F5F90932102923110F010922102909173
:10604000210280912202981729F48091F101806445
:106050008093F101559A0895DC0190910E02809190
:106060000D02981719F480E090E00895E92FF0E010
:10607000EE50FE4F80818C93892F8F5F80930E02AC
:106080008B3118F481E090E0089510920E0281E0C7
:1060900090E00895209121022E5F3091220222315A
:1060A00038F080E090E0332349F481E090E00895F7
:1060B00080E090E0231711F481E090E0089520E063
:1060C00030E09091220280912102981711F421E092
:1060D00030E0C9010895EF92FF920F931F93CF9381
:1060E000DF93CDB7DEB722970FB6F894DEBF0FBEB1
:1060F000CDBF1A8219827E010894E11CF11C46C0B2
:106100008BB78F7B8BBFC49886E00E94BB10C49A6C
:106110008BB780648BBF8BB78F7B8BBFC49882E0BB
:106120000E94BB10F70181810E94BB1089810E94EF
:10613000BB1000E010E089819A81800F911F885F79
:106140009F4340F480E00E94BB100F5F1F4F00345C
:10615000110589F7C49A8BB780648BBF00E010E00B
:106160001CC0C49A8BB780648BBF0AC0C49A8BB71B
:1061700080648BBF0F5F1F4F2EE2003E120769F451
:1061800089819A81805C9F4F9A83898389819A81D2
:106190008050904408F4B4CF0DC08BB78F7B8BBF79
:1061A000C49885E00E94BB1080E00E94BB1080FD77
:1061B000DDCFD7CF22960FB6F894DEBF0FBECDBF8E
:1061C000DF91CF911F910F91FF90EF900895EF9283
:1061D000FF920F931F93CF93DF937B018C0193E08A
:1061E000000F111F9A95E1F78BB78F7B8BBFC49877
:1061F00083E00E94BB10812F99270E94BB10802F43
:106200000E94BB10C0E0D0E087010C0F1D1F80E092
:106210000E94BB10F80180832196C830D105A1F7F8
:10622000C49A8BB780648BBF80E090E0DF91CF9100
:106230001F910F91FF90EF900895EF92FF920F93AF
:106240001F93CF93DF937B018C0133E0000F111F6D
:106250003A95E1F78BB78F7B8BBFC49886E00E949D
:10626000BB10C49A8BB780648BBF8BB78F7B8BBFFF
:10627000C49882E00E94BB10812F99270E94BB1016
:10628000802F0E94BB10C0E0D0E0F701EC0FFD1F93
:1062900080810E94BB102196C830D105B1F7C49A05
:1062A0008BB780648BBFC0E0D0E013C0C49A8BB7BB
:1062B00080648BBF80E090E019C0C49A8BB7806483
:1062C0008BBF21968EE2C03ED80719F48FEF9FEF67
:1062D0000DC08BB78F7B8BBFC49885E00E94BB102D
:1062E00080E00E94BB1080FDE8CFE0CFDF91CF912E
:1062F0001F910F91FF90EF9008959091E906969568
:106300009093E9068091E80680FF03C0906890931F
:10631000E9069091E80696959093E8068091E70645
:1063200080FF03C090689093E8068091E706869509
:106330008093E70686FF03C080688093E706089590
:10634000E82FF0E0EE0FFF1FEB5CFD4F80819181A5
:10635000009719F00197918380830895BF92CF929F
:10636000DF92EF92FF920F931F93CF93DF93082F4B
:10637000C82EDD24F601EB50F94F108123E0B22E38
:10638000B80E8B2D0E949810E601CC0FDD1F8430D3
:1063900098F48DE70E94330822E030E00C2E02C012
:1063A000220F331F0A94E2F7F82EF2228DE70E94A3
:1063B000330821E030E012C08DE70E94330821E06D
:1063C00030E00C2E02C0220F331F0A94E2F7F82EA1
:1063D000F2228DE70E94330822E030E002C0220F53
:1063E000331FCA95E2F78223E02EE294EE0CB0EE62
:1063F000EB22113019F5F601EE0FFF1FEB5CFD4F9C
:106400001182108285E1E82AE092E10666EE76E0EC
:1064100081EE96E00E94EF04F601EE5CFD4F809164
:10642000E806808362E0802F0E9415098B2D0E9470
:106430009810823008F4B8C112E0B7C1123051F49C
:10644000802F8A5F0E949810682F802F0E948F09EA
:1064500013E0ABC1133021F4882309F0A5C1A5C115
:10646000143051F4802F8A5F0E949810682F802F7B
:106470000E94720915E099C1153089F4FF2009F4D2
:1064800094C1802F0E946709F601EE0FFF1FEB5C9D
:10649000FD4F8EE190E09183808316E086C1163037
:1064A000A1F4F601EE0FFF1FEB5CFD4F808191819F
:1064B000892B09F07AC1802F875F0E949810682F7E
:1064C000802F0E948F0917E070C11730D9F4FF2088
:1064D00009F06BC122E043E060E08E2D84610E94F0
:1064E000E90520E040E060E08E2D8C610E94E90526
:1064F000802F875F0E949810682F802F0E9472095A
:1065000018E053C1183011F5FF2009F44EC1802F57
:106510000E9467098E2D8D618093E10666EE76E01C
:1065200081EE96E00E94EF042091E9064091E80692
:106530006091E7068E2D0E94E90520E043E060E0CF
:106540008E2D84610E94E90519E02FC1193009F0F0
:1065500041C08DE78093E10666EE76E081EE96E03D
:106560000E94EF048091E60690E09601220F331F0F
:1065700002C0959587952A95E2F780FF16C18B2D6D
:106580000E949810182F62E0802F0E941509802F1A
:106590000E94670920E040E060E08E2D0E94E9053E
:1065A00020E040E060E08E2D82600E94E90513301B
:1065B00039F08091240290912502892B09F473C04F
:1065C000802F875F0E949810682F802F0E94720989
:1065D0001AE0EBC01A3061F4FF2009F4E6C020E0B5
:1065E00040E060E08E2D8C610E94E9051BE0DDC07B
:1065F0001B3009F05AC0FF2009F0D7C0802F0E943D
:1066000067098E2D8D618093E10666EE76E081EE5E
:1066100096E00E94EF040E947D312091E9064091AE
:10662000E8066091E7068E2D0E94E90520E043E030
:1066300060E08E2D84610E94E9051091E9061095B5
:106640001093E9060091E80600950093E806F090A3
:10665000E706F094F092E7060E947D318091E9060A
:10666000810F8093E906882329F48091E8068F5FE3
:106670008093E8068091E806800F8093E8068823DF
:1066800029F48091E7068F5F8093E7066091E70623
:106690006F0D6093E7062091E9064091E8068E2D84
:1066A0008A610E94E9051EE080C01E3009F06EC0BC
:1066B0008091E60690E09601220F331F02C0959567
:1066C00087952A95E2F780FF70C062E0802F0E94D4
:1066D0001509802F0E9467098B2D0E949810833026
:1066E00031F08091240290912502892B91F0109233
:1066F000E6061092E7061092E806F601EE0FFF1F7D
:10670000EE0FFF1FEA5DFD4F10821182128213828D
:1067100003C08E2D0E944E0B2091E9064091E806A1
:106720006091E7068E2D0E94E9051E2D12602091D2
:10673000E9064091E8066091E706812F0E94E9058D
:1067400020E040E060E08E2D0E94E90520E040E07E
:1067500060E0812F0E94E905F601EE5CFD4F20E02C
:10676000408160E08E2D84610E94E905F601EE0F04
:10677000FF1FED59F84F40815181662757FD609505
:10678000762F8E2D86600E9431090CC01F3069F46F
:10679000F601EE5CFD4F22E0408160E08E2D8461C9
:1067A0000E94E90510E001C014E0E5EFF6E0CE0E2E
:1067B000DF1EF6011083DF91CF911F910F91FF90A3
:1067C000EF90DF90CF90BF900895AC018091AB0423
:1067D000882319F480E090E008958BB78F7B8BBFFE
:1067E00090913C0280913B02981711F490E01EC0FA
:1067F00020913C02822F90E0FC0134E0EE0FFF1F5D
:106800003A95E1F7E81BF90BDA01E559FC4F8FE007
:1068100001900D928150E1F72F5F20933C0280910F
:106820003C02843111F410923C0291E08BB78064F9
:106830008BBF892F90E008950F931F93CF93DF9321
:10684000DA9895E090939704809398046093990464
:1068500040939A04C0E0D0E08E0109561B4FF80126
:1068600080810E94BB10F80180832196C430D1053D
:1068700099F7DA9ADF91CF911F910F910895EF92D6
:10688000FF920F931F93CF93DF93DA9892E0909348
:10689000970480939804EE24FF24C62FD0E022961C
:1068A00009C08C0109561B4FF80180810E94BB1062
:1068B000F80180838E2D90E00894E11CF11C8C1768
:1068C0009D077CF3DA9ADF91CF911F910F91FF9092
:1068D000EF9008950F931F93CF93DF93DA9892E090
:1068E000909397048093980460939904C0E0D0E05B
:1068F0008E0109561B4FF80180810E94BB10F801E0
:1069000080832196C330D10599F7DA9ADF91CF9130
:106910001F910F910895EF92FF920F931F93CF93C2
:10692000DF93DA9893E09093970480939804EE2491
:10693000FF24C62FD0E0229609C08C0109561B4FB8
:10694000F80180810E94BB10F80180838E2D90E0B9
:106950000894E11CF11C8C179D077CF3DA9ADF91F7
:10696000CF911F910F91FF90EF900895EF92FF92BA
:106970000F931F93CF93DF93EC017A018B01109259
:106980003E0280913E0280933D0280913D028093C1
:106990003C0280913C0280933B0264E88FE00E94BD
:1069A0006A3461E08EE00E948B34809199048F3FBD
:1069B00019F41092AB049AC08091990487FFF1CF2B
:1069C00081E08093AB04C130D10511F467E211C0BE
:1069D000C230D10551F46FE08AE20E946A346FEB55
:1069E00089E20E946A3467E038C0C330D10531F4CF
:1069F00067E08AE20E946A346AEBF2CFC430D105C4
:106A000011F463E0F6CFC530D10511F463E011C095
:106A1000C630D10551F463E08AE20E946A3468E925
:106A200089E20E946A3461E018C0C730D10551F490
:106A300060E08AE20E946A3468EB89E20E946A346C
:106A400065E00BC0289761F460E08AE20E946A3436
:106A500060E989E20E946A3462E088E20E946A3456
:106A600060E08DE00E946A3460E08CE00E946A344D
:106A7000D801C70143E0B695A795979587954A95A4
:106A8000D1F7809399048E2D8295880F807E809314
:106A90009A0410929B0410929C0464E080E00E948F
:106AA0003F348FEF8093990480EE80939A04109284
:106AB0009B0410929C0464E080E20E943F3460E0FA
:106AC00080E60E946A3461E18BE20E946A3464E0ED
:106AD0008FE00E946A3461E08EE00E948B348091E6
:106AE000990487FDF8CF8BB780648BBFDF91CF917E
:106AF0001F910F91FF90EF900895AC018091AB042E
:106B0000882319F480E090E008958BB78F7B8BBFCA
:106B100020913D022F5F243109F420E080913E0254
:106B2000281711F490E023C080913D0290E0FC0111
:106B300064E0EE0FFF1F6A95E1F7E81BF90BE15CDB
:106B4000FD4FDA018FE00D9001928150E1F7209323
:106B50003D0261E080E50E948B348091990483FDC1
:106B600005C040E160E18CE20E941C3491E08BB7EB
:106B700080648BBF892F90E008951F920F920FB60B
:106B80000F921124EF92FF921F932F933F934F93F5
:106B90005F936F937F938F939F93AF93BF93CF93A5
:106BA000DF93EF93FF9361E08CE20E948B3480913E
:106BB0009904E82E80FFC1C010913B021F5F143181
:106BC00009F410E080913C02181709F4B1C09091CB
:106BD0003B028FE0989FE0011124C559DC4F6EE025
:106BE00080E60E948B3480919B04869586958695DD
:106BF000817089838981882309F45AC080919E0419
:106C000082958695869581708A8380919B0490E019
:106C1000A0E0B0E0FBE1880F991FAA1FBB1FFA9507
:106C2000D1F78B839C83AD83BE832B813C814D81C7
:106C30005E8180919C0490E0A0E0B0E0E3E1880FE9
:106C4000991FAA1FBB1FEA95D1F7822B932BA42B68
:106C5000B52B8B839C83AD83BE832B813C814D817F
:106C60005E8180919D0490E0A0E0B0E0072E7BE083
:106C7000880F991FAA1FBB1F7A95D1F7702D822B01
:106C8000932BA42BB52B8B839C83AD83BE832B814D
:106C90003C814D815E8180919B04829586958770B1
:106CA00090E0A0E0B0E0822B932BA42BB52B0FC07B
:106CB0008091990486958695869581708A838091C6
:106CC0009B0482958695877090E0A0E0B0E08B836E
:106CD0009C83AD83BE832B813C814D815E818091FD
:106CE0009A0490E063E0880F991F6A95E1F7AA275C
:106CF00097FDA095BA2F822B932BA42BB52B8B83BA
:106D00009C83AD83BE8380919E048F70888320E036
:106D100030E0F901E156FB4F8081F901EC0FFD1FD6
:106D200087832F5F3F4F2830310599F710933B023F
:106D300040E061E08CE20E941C34E4FE96C040E03A
:106D400060E18CE20E941C3490913E0280913D02F1
:106D5000981709F48AC080913E029FE0899FE00164
:106D60001124C15CDD4F8F5F80933E028B819C813B
:106D7000AD81BE8113E0B695A795979587951A9535
:106D8000D1F7809399048B819C81AD81BE818295DE
:106D9000880F807E80939A0489818823C9F180912D
:106DA0009A04886080939A0420919A048B819C8134
:106DB000AD81BE81FBE1B695A79597958795FA952C
:106DC000D1F78370822B80939A0420919B048B814E
:106DD0009C81AD81BE81E3E1B695A7959795879596
:106DE000EA95D1F7282B20939B0420919C048B815A
:106DF0009C81AD81BE81072E7BE0B695A7959795C6
:106E000087957A95D1F7702D282B20939C0404C088
:106E100010929B0410929C0488818F7080939D0433
:106E20008A81882329F080919D04806480939D0449
:106E300020E030E0F901EC0FFD1F8781F901E256F7
:106E4000FB4F80832F5F3F4F2830310599F76DE06E
:106E500081E50E943F346BE080E50E946A348091B6
:106E60003E02843111F410923E02FF91EF91DF91C6
:106E7000CF91BF91AF919F918F917F916F915F91D2
:106E80004F913F912F911F91FF90EF900F900FBE68
:106E90000F901F901895823010F482E001C08E7F11
:106EA00082B985EC86BF85B3836085BB0895DC011C
:106EB0009091AC04961719F080E090E0089540E0BE
:106EC00020E030E00BC0F901E155FB4F8081FD016E
:106ED000E20FF31F80834F5F2F5F3F4F491799F7F2
:106EE0001092AC0481E090E00895DC0140E020E0E5
:106EF00030E00BC0FD01E20FF31F8081F901E8547F
:106F0000FB4F80834F5F2F5F3F4F461799F760938A
:106F1000AE0408951F920F920FB60F9211248F9313
:106F20009F93EF93FF9381B1803629F485EC86BF60
:106F30001092AC0453C081B1803819F081B1883807
:106F400071F485EC86BF8091AC04E82FF0E093B13A
:106F5000E155FB4F90838F5F8093AC043FC081B1BC
:106F6000803AD1F181B1882311F485ED36C081B129
:106F7000883AB1F41092AD049091AD04E92FF0E09D
:106F8000E854FB4F808183B99F5F9093AD0485ECFB
:106F900086BF9091AD048091AE049817F9F416C0A5
:106FA00081B1883BC9F49091AD04E92FF0E0E85439
:106FB000FB4F808183B99F5F9093AD0485EC86BFC2
:106FC0009091AD048091AE04981741F48091AD0486
:106FD00081508093AD0402C085EC86BFFF91EF9194
:106FE0009F918F910F900FBE0F901F901895FF9259
:106FF0000F931F93982F162F042FF22E8091C10408
:10700000813029F48BB78F7B8BBFAF980DC0823056
:1070100029F48BB78F7B8BBFAE9806C0833021F4E9
:107020008BB78F7B8BBFAD98892F0E94BB10812FB0
:107030000E94BB10802F0E94BB108F2D0E94BB109E
:1070400085B3806E85BB8BB780648BBF1F910F911A
:10705000FF900895CF93DF93CDB7DEB724970FB697
:10706000F894DEBF0FBECDBF49835A836B837C8308
:10707000813011F48AE005C0823011F48CE001C047
:1070800088E029814A816B8181600E94F7372496CC
:107090000FB6F894DEBF0FBECDBFDF91CF9108953C
:1070A000CF93DF93CDB7DEB724970FB6F894DEBF4A
:1070B0000FBECDBF882311F4E0E005C0813011F48C
:1070C000E2E001C0E4E0842F90E09695982F8827B5
:1070D00097958795A0E0B0E09B0140E050E06CE020
:1070E000220F331F441F551F6A95D1F7822B932B14
:1070F000A42BB52B89839A83AB83BC8329814A81D6
:107100006B818E2F81600E94F73724960FB6F8941A
:10711000DEBF0FBECDBFDF91CF91089520E040E0EC
:1071200064E087E00E94F73720E040E060E281E120
:107130000E94F73720E040E060E089E00E94F737E6
:1071400020E040E060E08BE00E94F73720E040E084
:1071500060E08DE00E94F7370895CF92DF92EF92C2
:10716000FF920F931F93CF93DF936C017B0180916C
:10717000C104813029F48BB78F7B8BBFAF980DC0D2
:10718000823029F48BB78F7B8BBFAE9806C08330DB
:1071900021F48BB78F7B8BBFAD98C0E0D0E0870127
:1071A0000C0F1D1FF601EC0FFD1F80810E94BB100C
:1071B000F80180832196C430D10589F785B3806EAC
:1071C00085BB8BB780648BBFDF91CF911F910F91EF
:1071D000FF90EF90DF90CF900895CF93DF93CDB7DE
:1071E000DEB72C970FB6F894DEBF0FBECDBF81304F
:1071F00011F48AE005C0823011F48CE001C088E00F
:107200008D83BE016F5F7F4FCE0105960E94AD3822
:107210001C868A818B879B819A879C81998787FFAF
:1072200003C08FEF8C8701C01C8669857A858B85AA
:107230009C852C960FB6F894DEBF0FBECDBFDF91B4
:10724000CF9108958091C6049091C704FC0105C0B8
:107250002C3211F4108204C0319620812223C1F710
:107260003196F093C704E093C6040895CF92DF925D
:10727000EF92FF920F931F93CF93DF93CDB7DEB7BB
:1072800064970FB6F894DEBF0FBECDBF6B017C01D3
:107290000E945F308823E1F380E20E9410302AE0F0
:1072A00030E08E010F5F1F4FA801C701B6010E9499
:1072B000833CEE24FF2468010DC00E944A308823DD
:1072C000E1F70C0D1D1DF80180810E94103008941B
:1072D000E11CF11C0E2D10E0F601E00FF11F808182
:1072E000882359F764960FB6F894DEBF0FBECDBF62
:1072F000DF91CF911F910F91FF90EF90DF90CF9092
:1073000008950F931F93CF93DF93CDB7DEB72497E4
:107310000FB6F894DEBF0FBECDBF8C010E945F3068
:107320008823E1F3F8018081805C0E941030F8012D
:107330008181805C0E941030F801628170E080E001
:1073400090E00E943639F80184818C8385818B839B
:1073500086818A838781898369817A818B819C81F7
:107360000E9436398DE00E94103024960FB6F894B2
:10737000DEBF0FBECDBFDF91CF911F910F9108955A
:10738000CF92DF92EF92FF920F931F93CF93DF93F1
:10739000EC0101C021961881812F90E00E944A3DA6
:1073A000892BC1F71D3229F4219681E0C82ED12CFA
:1073B00005C01B3209F42196CC24DD2420E030E006
:1073C00040E050E01AC0FF2400E010E080ED9FEFA5
:1073D000AFEFBFEFE80EF91E0A1F1B1FCA01B9016C
:1073E0002AE030E040E050E00E94C73C9B01AC0145
:1073F0002E0D3F1D401F511F2196E8808E2D90E0DD
:10740000C0970A9700F3CD2839F0509540953095F4
:1074100021953F4F4F4F5F4FCA01B901DF91CF9187
:107420001F910F91FF90EF90DF90CF9008958F9272
:107430009F92AF92BF92CF92DF92EF92FF920F9303
:107440001F93CF93DF93CDB7DEB725970FB6F89490
:10745000DEBF0FBECDBF5C01CE0101960E942C3075
:10746000882309F4FAC08091C3048823A9F509810F
:1074700010E082E090E00E94111090E0805C9F4F4D
:107480000817190789F48091C4049091C504892BC9
:1074900009F0E3C081E08093C304809163018823F5
:1074A00009F0DBC08981D7C089818D3011F08B3123
:1074B00029F41092C5041092C404CFC08091C40472
:1074C0009091C5048F37910508F0C7C0019690933D
:1074D000C5048093C404C1C080916301882319F45A
:1074E00089810E9410302981203268F08091C40483
:1074F0009091C5048F379105A8F4FC01E853FB4F28
:10750000208301960AC0283069F48091C4049091C8
:10751000C504009709F491C001979093C504809326
:10752000C4048BC02D3009F088C08091C4049091B0
:10753000C504892B09F481C080916301813021F554
:107540000E945F308823E1F382E090E00E941110F6
:10755000805C0E94103000E010E00CC00E944A30B5
:107560008823E1F7F801E853FB4F80810E94103037
:107570000F5F1F4F8091C4049091C504081719072D
:1075800068F38DE00E9410301092C7051092C60576
:107590002091C4043091C5046091C6047091C70461
:1075A00048EC54E090E0A0E0B0E0240F351F2EC07E
:1075B000913081F0913018F0923031F51CC0FA0111
:1075C0008081803209F1FD01E95BFA4F80831196D9
:1075D00091E01AC0FA018081803289F4A230B105AD
:1075E00028F0FD01E95BFA4F10821196BD01695B3D
:1075F0007A4F92E009C0FA018081803229F0FD01C2
:10760000E95BFA4F808311964F5F5F4F4217530734
:1076100079F67093C7046093C604B093C705A0932E
:10762000C605A95BBA4F1C9281E08093C2041092F8
:10763000C3041092C5041092C40489818B3169F48B
:107640001092C5041092C4041092C3048091630187
:10765000882319F48DE00E9410308091C2048823A1
:1076600019F480E090E0BCC01092C204CC24DD2468
:1076700027E4822E25E0922E760193E0EE0CFF1C8B
:107680009A95E1F7EC18FD08870100571E4FB801E5
:10769000C4010E94703C892B61F4F701EB56FE4F48
:1076A0008491F701EA56FE4FE491982F3E2F21E096
:1076B0000EC0F8018491882339F00894C11CD11CB4
:1076C000FFEFCF16D104C1F620E090E030E0D50105
:1076D00081E0FD0111828F5F11968830D1F722235E
:1076E00009F461C0D5019C93E32E30FF40C00E9495
:1076F00022398C01F50180818430A1F465E872E0C3
:10770000C8010E94703C892BB1F061E872E0C801A9
:107710000E94703C892BC9F06BE772E0C8010E949F
:10772000703C1AC08D30F1F465E772E0C8010E9428
:10773000703C892B19F4F501118219C060E772E0E1
:10774000C8010E94703C892B11F481E008C069E6F1
:1077500072E0C8010E94703C892B21F482E0F5019F
:10776000818305C0C8010E94C039F5016183E1FE33
:1077700006C00E9422390E94C039F5016283E2FEF0
:1077800015C00E9422390E94C0396A837B838C8392
:107790009D838D81F50183838C8184838B81858397
:1077A0008A81868303C08FEFD5018C938501095FA1
:1077B0001F4F82E090E00E941110F501878320E0C6
:1077C00030E0F501E20FF31FD8018C919081890F11
:1077D0008C932F5F3F4F2730310599F781E090E080
:1077E00025960FB6F894DEBF0FBECDBFDF91CF91C7
:1077F0001F910F91FF90EF90DF90CF90BF90AF90CF
:107800009F908F900895A0E0B0E0E9E0FCE30C9435
:10781000713DEC01688179818A819B8161157105D7
:107820008105910549F484E2A82E89EDB82E8BE5F7
:10783000C82E87E0D82E02C05B016C01C601B501DD
:107840002DE133EF41E050E00E940D3D27EA31E4A5
:1078500040E050E00E94C73C7B018C01C601B501AD
:107860002DE133EF41E050E00E940D3DCA01B90126
:1078700024E13BE040E050E00E94C73CE61AF70AF2
:10788000080B190B17FF08C08FEF9FEFAFEFBFE793
:10789000E80EF91E0A1F1B1FE882F9820A831B8368
:1078A0008FEF9FEFAFEFBFE7E822F9220A231B23F8
:1078B000C801B701EAE0CDB7DEB70C948D3D0E9458
:1078C000033C08958FE091E00E94033C089560938B
:1078D0000F0170931001809311019093120108958C
:1078E000FB01DC018D9181341CF08B350CF4805E42
:1078F000659161341CF06B350CF4605E861B611180
:1079000089F3990B0895FA01CF93FF93EF932230F7
:1079100044F1253234F5C22FE894CA3049F497FB7C
:107920003EF490958095709561957F4F8F4F9F4F56
:107930002C2F332744275527FF93EF930E94283D90
:10794000EF91FF91605D6A330CF0695D6193B9015D
:10795000CA01605070408040904051F716F4CDE26B
:10796000C19310828F919F91CF910C94B73CDC0111
:10797000FC01672F71917723E1F7329704C07C9166
:107980006D9370836291AE17BF07C8F30895629F2D
:10799000D001739FF001829FE00DF11D649FE00D07
:1079A000F11D929FF00D839FF00D749FF00D659F68
:1079B000F00D9927729FB00DE11DF91F639FB00D67
:1079C000E11DF91FBD01CF0111240895AA1BBB1BA6
:1079D00051E107C0AA1FBB1FA617B70710F0A61BCF
:1079E000B70B881F991F5A95A9F780959095BC01F0
:1079F000CD01089597FB092E07260AD077FD04D004
:107A0000E5DF06D000201AF4709561957F4F089548
:107A1000F6F7909581959F4F089597FB092E0526BF
:107A20000ED057FD04D014D00AD0001C38F4509565
:107A30004095309521953F4F4F4F5F4F0895F6F792
:107A400090958095709561957F4F8F4F9F4F0895CA
:107A5000A1E21A2EAA1BBB1BFD010DC0AA1FBB1F52
:107A6000EE1FFF1FA217B307E407F50720F0A21BC4
:107A7000B30BE40BF50B661F771F881F991F1A9431
:107A800069F760957095809590959B01AC01BD015B
:107A9000CF01089591111AC0803219F08950855094
:107AA000D0F70895E199FECFBFBBAEBBE09A119627
:107AB0000DB20895E199FECFBFBBAEBB0DBA1196D2
:107AC0000FB6F894E29AE19A0FBE08959927882795
:107AD00008952F923F924F925F926F927F928F9272
:107AE0009F92AF92BF92CF92DF92EF92FF920F934D
:107AF0001F93CF93DF93CDB7DEB7CA1BDB0B0FB657
:107B0000F894DEBF0FBECDBF09942A883988488813
:107B10005F846E847D848C849B84AA84B984C884A9
:107B2000DF80EE80FD800C811B81AA81B981CE0FA0
:107B3000D11D0FB6F894DEBF0FBECDBFED01089585
:027B4000FFCF75
:107B4200141414D41187253D254D1B162EA526D5B8
:107B52002214224B21461F931D6E1C571B031B2010
:107B620029A428D611D811DA11DC1101144814CD38
:107B720014D614F21405150C15D71913151319B0D0
:107B82001854181D26D91285282C21161551155E58
:107B9200155F15611563156515671569156B156D0B
:107BA200156F15711573157515771579157B157D7B
:107BB200157F15811583158515871589158B158DEB
:107BC200158F152C0433042D042E042F0430043198
:107BD20004320491159415A415A815DE17CD15B31A
:107BE20017D4158A17A01824163A16F0164816014B
:047BF200000000008F
:00000001FF
